:020000040800F2
:10000000D0240020D9000008AD180008A101000884
:1000100000000000000000000000000000000000E0
:10002000000000000000000000000000E5000008E3
:1000300000000000000000001F010008771D0008FC
:10004000EB000008EB000008F1180008EB000008C6
:10005000EB000008EB000008EB000008EB000008D4
:10006000EB000008D5080008310900080000000076
:10007000EB0000080000000000000000EB0000089A
:10008000EB000008EB000008EB000008EB000008A4
:10009000EB000008EB00000800000000EB00000887
:1000A000EB000008BD1F0008EB000008EB00000893
:1000B000F9160008EB000008EB000008EB00000850
:1000C0000448854600F0A0F900F012F90048004706
:1000D00005050008D0240020044880470448004754
:1000E000FEE7FEE7FEE7FEE7FEE7FEE70D1E00087F
:1000F000C1000008EFF3108072B6704780F31088DB
:1001000070472A4A1368012B03D001231360284A41
:100110001060284A11602848284901607047EFF3B1
:10012000108272B62148016800291DD000210160AB
:100130001F48016800290AD0EFF3098120390068BF
:100140000160F0C144464D4656465F46F0C119492C
:1001500009680968F0C9F0B4F0C9A046A946B246DA
:10016000BB46F0BC81F3098882F31088042040422A
:100170000047104908600E49002008600B49012023
:1001800008600F480F490268114301600A480B4993
:1001900001600D480068006880F3088862B6704707
:1001A000EFF3098000B504F071FD00BD8413002059
:1001B0005C1000206010002004ED00E00000001042
:1001C00020ED00E00000FFFF08ED00E0F0B51FB4F7
:1001D0000646002082B005464024019100901BE0B5
:1001E000019922460F46304600F0C5F8049A059B57
:1001F000801A994110D310461946224600F0ABF8F8
:10020000361A8F410197224601200021009F00F0FD
:10021000A2F838184D4100902046641E0028DFDC0B
:10022000019B00982946324607B0F0BD03460B43B8
:100230009B0703D009E008C9121F08C0042AFAD29C
:1002400003E00B780370401C491C521EF9D2704722
:10025000D2B201E00270401C491EFBD2704700225E
:10026000F6E710B513460A4604461946FFF7F0FFB5
:10027000204610BD10B5044605E00B780370401C05
:10028000002B00D0491C521EF7D2204610BD421C44
:100290000178401C0029FBD1801A704730B5044614
:1002A0000020034600E05B1C934203D2E05CCD5C7F
:1002B000401BF8D030BD30B505460020034600E0B5
:1002C0005B1C934205D2EC5CC85C201A01D1002C67
:1002D000F6D130BD70B5064607F01CFC0468054633
:1002E0000A220021304600F057F82C6070BD000053
:1002F0007CB507480090074801900546009C04E043
:100300002046016808188047241DAC42F8D17CBD06
:100310008C9700089097000870B50446002903D018
:1003200000202022012310E0002801D00020C0433B
:10033000C046C0460DE02546D5408D4205D30D464A
:100340009540641B1D46954040191546521E002DD0
:10035000F1DC214670BD10B5202A04DB0146203AAD
:100360009140002010BD914020239C1A0346E34099
:100370001943904010BD10B5202A04DB0846203AEE
:10038000D040002110BD0B46D340D0402024A21AFB
:1003900091400843194610BDF7B5009C0F46002652
:1003A0002578641C002D05D000F046F80068405DFB
:1003B000C007F5D12B2D02D02D2D18D0641E394643
:1003C0002046029A00F03CF8002F04D03968A14280
:1003D00001D1009939607105022400290BDA4042ED
:1003E000002803DD07F096FB0460A007FEBD012096
:1003F00080020643E3E70028F8DA07F08BFB04608D
:100400000048FEBDFFFFFF7F1CB50948009009486A
:10041000019005460126009C05E0E36807CC3343C4
:100420000C3C98471034AC42F7D3FFF74DFE000068
:100430006C9700088C97000800487047BC7B000848
:10044000F7B582B0029C00272078641C15460197FE
:10045000302802D0002D15D015E020780127641C2B
:10046000782804D0582802D0002D09D00BE0002DA8
:1004700001D0102D07D1002710252078641C02E040
:10048000082500E00A250026009610E000990127C3
:1004900069430818020C294680B2714300908E18F7
:1004A0003804864201D3012001902078641C29463B
:1004B00000F019F80028E9DA0398002805D0002F89
:1004C00001D0641E00E0029C04600198002806D060
:1004D00007F020FB02210160C81E05B0F0BD0099A5
:1004E00030040843F9E73A2800D230382023024686
:1004F0009A43412A01D310463738884201D300205D
:10050000C043704780B506F039FC002080BD000074
:10051000F8B500241048114E062C16D0075D0025B2
:10052000AF4207D0305D281800F024FA6D1C002877
:10053000F6D002E0641C0848EEE70948009000206D
:1005400008A1434A434B01F0B5FA062C01D3002021
:10055000F8BD0120F8BDC046967D00089D7D0008CD
:10056000A3850008202025732573466C6173685F9E
:100570004572617365506167655F5265636F726450
:1005800073206661696C65640D0A0D0A25730000AD
:10059000F0B5FFB086B0214801680020204DA94287
:1005A00039D0029005A8049014307B218900FFF710
:1005B00056FE0595042003900090FD20C7000124FD
:1005C000022603253846214632462B4601F078F9AB
:1005D0000690039800900A373846214632462B464B
:1005E00001F06EF9322109910A2108910790FFF775
:1005F0008FFF00F0FBF9049800F0DAFC002809D026
:1006000008480090002008A1114A124B01F052FA4C
:10061000204600E002987FB006B0F0BD00FE000862
:10062000A5A4A3A2A3850008202025732573466CEA
:100630006173685F57726974655F436F6E6669675F
:10064000496E666F206661696C65640D0A257300EA
:10065000A885000889850008F8B5012481256D1E4C
:1006600010D00E1D071D096800F016FC002400289C
:1006700031463846F3D003200349012403A3224620
:1006800007F06EF9E0B2F8BD918500084253505F63
:10069000466C6173685F50726F6772616D5F496E1F
:1006A000666F50616765206661696C656400000073
:1006B000BFB5164800210A4605F074F914490860D0
:1006C000002805D103201349012213A307F048F99C
:1006D000052003900A200290154800900320400254
:1006E0000190144D14A1174A00242846234605F012
:1006F000BFFD284605F07EFE06200649012212A312
:1007000007F02EF9204604B0B0BDC046668500084B
:10071000A00800207085000868725F72785F7365BA
:100720006D20637265617465206661696C65640043
:1007300034090020A408002068725F746872656143
:10074000640000002D1600084253505F48525F4974
:100750006E697400BFB506F0D1FA134DCA20286047
:100760005320286000F08CF8104805F0BFFD0120F0
:10077000C003FF21EC3100F01DF800F091F80024D7
:100780002C60052003210091019002902420082173
:100790002322142300F026F80549C81C00F03CF879
:1007A000204604B0B0BDC04624280040B80B00006D
:1007B0009000002010B501225303094AD4681C435D
:1007C000D4601368DB03FCD40143D161FF20000433
:1007D0003E490A6882430A603D480421016010BD19
:1007E0000C2800401CB51C466B46D8709A70597096
:1007F00006981870184606F017FD002800D0FEE78E
:100800000599049A01A881704270047006F064FD95
:10081000002800D0FEE71CBDFFB500910190072025
:100820000006029004231449029D144E5B1E21D041
:100830000F684A680C684868A742F7D114460F4908
:100840000C40D102294021430392C20230402A4089
:1008500002439142039A0849E8D100998F70380AFF
:100860004870380C087001998A70200A4870100C82
:100870000870FFBDFEE7C04600280040FF1FFFFFD5
:100880000720400505490A68824301204305D21824
:100890000A60C0040A6802430A60704718280040D2
:1008A0000948CA21016153210161016804221143F1
:1008B000016000210161FF20000404490B688343AB
:1008C0000B600348026070471428004000E400E019
:1008D00000E100E010B504F097FA244CA06840074E
:1008E0000AD52068400707D560680421014361608C
:1008F0001F48406805F0AEF8A06880070AD5206858
:10090000800707D56068022101436160184840688C
:1009100005F0A0F8A068000706D52068000703D5F9
:10092000606808210143616004F088FA10BDC04688
:1009300010B504F069FA0D48C169890712D501683C
:1009400089060FD5C16902229143C1614168202205
:100950000A434260064CA1682046383003F09DFAF5
:100960000020A06004F06AFA10BDC04600000240FA
:1009700030010020BCB50446104DE868002803D5BE
:100980000F4828600F4828600F480094019000200D
:100990000EA1144A144B01F08DF800F051F9022019
:1009A000214606F083FA044600F050F90120C00702
:1009B000E9680143E9602046BCBDC046082002400A
:1009C000851A7AE591836E7CA38500082020257323
:1009D00025734572617365506167652025640D0A52
:1009E000257300009B85000885850008E0B57F2001
:1009F000FFF7C0FF002807D004480090002004A1A2
:100A00004C4A4D4B01F056F88CBDC046A3850008FA
:100A10002020257325736572726F725F7061676540
:100A2000203D202523780D0A0D0A257300000000C3
:100A3000F0B587B0002202604260049002928260AA
:100A40002E48425C039188002D490B5801202D4D02
:100A50000692C4B2944246D805900106CF0B7D1988
:100A60000422D11B8126B000C71B761E08D0281D8A
:100A7000091F3F1F121F5D596D1C0546F5D104E08B
:100A80000598401C069A1F4DE3E7D81B069DAC4213
:100A90000DD2591A0A68521C1DD0049A51609060F8
:100AA0005480039840001849085A108023E0991A8E
:100AB000049A516090605480039840001249085A8B
:100AC0001080012C17D11146536093601868401CA8
:100AD00011D1029805E004994B6088604C807842FF
:100AE0008008088007E009480090002008A1D64A45
:100AF000D64B00F0DFFF07B0F0BDC046967D000882
:100B0000A47D000800FEFFFF887D0008A385000883
:100B1000202025732573466C6173685F47657449AF
:100B20006E6465785F506F73204572726F72210D2D
:100B30000A257300A8850008898500081FB50146AD
:100B400001AC2046FFF774FF207804B010BD000010
:100B5000F0B58BB0471E062F34D814460D46F9B2B7
:100B60000AAE30462A4600F079F87178B3783278C8
:100B7000160909960396009701951D06AD0E089576
:100B800006951B0259181F270F4004970F26164081
:100B9000002802D1FD20C000361802968805C50E37
:100BA000059507200949012209A306F0D9FE0898F6
:100BB00060712571E7700998A0706670300A207026
:100BC000002000E001200BB0F0BDC0469185000878
:100BD00028256429466C6173685F476574526563B4
:100BE0006F72645B25645D3A253034642D253032A4
:100BF000642D253032642C253032643A253032643D
:100C00000000000070B5044600250C4E2846B04791
:100C100020800120B04760800220B047207103206F
:100C2000B04760710420B047A0710520B047E07163
:100C30000620B0472072284670BDC0463D0B000814
:100C400080B5FFF757FA0449086080BD80B50248B7
:100C50000068FFF753FA80BDD40F0020F0B591B0C3
:100C600016460D4604460EA8FFF7E2FE68006349EB
:100C7000085A711E81420AD20EA80288B24219D2C5
:100C800060480096019202900025824905E05D4986
:100C900000960190029100255BA16B4A6B4B2846A0
:100CA00000F008FFE570A5706570257001252846E5
:100CB00011B0F0BDA80052490858B1000F9F8742FB
:100CC0000D920B9702D10818001F21E04A4A525D8D
:100CD0007B1852021018091F0C9183420DD9494804
:100CE00000970190002066490A92634A634B00F026
:100CF000E1FE0C980A99401A09E0424800970190D9
:100D0000002053A15C4A5D4B00F0D4FE0C98C01942
:100D10000C900768384601F01FF8390E884240D120
:100D20002770E170380CA0703A0A62703802800EA9
:100D30000A90B903C90E1F2313403A06120F0F2061
:100D40003840FD27FF00C0190095019602AD0DC582
:100D500005910A9806902B4E079600254B49464A66
:100D6000464F28463B4600F0A5FEE078A178227861
:100D700063780EAC64881B029A18090400064018B8
:100D800080180B9900910C9901910D99029103948F
:100D9000049005963E492846374A3B4600F08AFEB5
:100DA00085E70A910EA94A88164B09900B99009184
:100DB0000C9801900D9802A985C105930026314930
:100DC000214F224B30463A4600F074FE0D980090B9
:100DD0000195099802900A9803900C98049009488C
:100DE0000590294930463A46184B00F063FEE670FC
:100DF000A6706670267059E7967D0008887D000809
:100E0000A47D0008A3850008202025732573696E42
:100E1000646578206E756D2028256429203E206841
:100E200072207265636F7264206D6178206E756DDB
:100E300020256420262620696E646578203E2030B7
:100E40000D0A257300000000A885000889850008A8
:100E500020202573257372656164203A68725F7380
:100E6000746172745F6164647231203D202523785F
:100E70000D0A2573000000009B8500088585000889
:100E8000658A00084C87000819860008EE8900086A
:100E9000B88500087A890008F0B585B00446800757
:100EA0000AD0009403202349012523A32A4606F0F3
:100EB00057FD284605B0F0BD0E46264F1C20B860F1
:100EC000F868002803D52448386024483860F8685A
:100ED00000250028EDD40495FFF7B2FE20463146E8
:100EE00006F02AF80546FFF7B1FE002D0ED0206867
:100EF0000094019007200F49012519A32A4606F006
:100F00002FFDE807F9680143F960D2E70125E807FA
:100F1000F9680143F9602068B04204D1022005F06D
:100F2000E5F9049DC5E70094019602900720014968
:100F300010A3BBE7918500086164647220252358E3
:100F4000206973206E6F7420616C69676E65640D33
:100F50000A00000008200240851A7AE591836E7C21
:100F600061646472203D202523582C2072656164E1
:100F700020256400466C6173685F57726974652050
:100F800044617461204D69736D617463682061749C
:100F90002061646472202523582C20657870656375
:100FA00074656420256420676F7420256400000048
:100FB00080B501460148FFF74FFB80BD00FE0008E9
:100FC000F0B597B00446062816D179480068411C50
:100FD00012D0169077480127002406250095019429
:100FE000029703907449754A754B204600F062FDE4
:100FF00016A829462246D5E013A812902146FFF7ED
:1010000017FD16AE00201090F0706E490A78130993
:101010000A204343D21808320F231A401F464B7848
:1010200011941D094543EB181B019A183270664B49
:101030001A7815093C463A404543AD181F220F92D5
:1010400015400E956D015B781F09234022460B94D5
:101050004743FB183F241C400D94A3025B191C0A54
:101060000994B47089780F091140474378180F9993
:1010700008400C901C1874701298078840881290D1
:10108000149D15980890169800F066FE0A9009992C
:10109000B17011997470F070169E464809950095CC
:1010A000089C01940F970297129A03920D4604969A
:1010B00005904649464A474B109F384600F0FAFCD7
:1010C0003006000F0B9A3240FD21C90051180095DF
:1010D000019102900C9803900E9804900D98059041
:1010E0000A980690334807903B493846384A394BAE
:1010F00000F0E0FC254620463146FFF7CDFE0028F3
:101100001BD02C480090002434A12C4F2C4B20469F
:101110003A4600F0CFFC0998009001950F98029094
:1011200012980390049623480590344920463A4685
:10113000234B00F0BFFC012736E00F9E1198800082
:101140002F490858129949020818001F85421FD1DB
:1011500000951848019000202A492B4A2B4B00F09B
:10116000A9FC2B481199445C2A48405C12998142A1
:1011700001D2129824182046FFF7FCFB002807D064
:1011800000940C480190002023491F4A1F4BD0E7D0
:10119000119840002149085A3246864200D2521C1A
:1011A00016A81199FFF75AFD384617B0F0BDC04692
:1011B00000FC0008A38500080B870008A88500082C
:1011C000898500089300002090000020EC8700082B
:1011D0009B85000885850008A488000820202573C9
:1011E000257368725F77726974655F646174615FAB
:1011F0006572726F720D0A25730000004B8800083B
:10120000A47D0008EF880008B08500088D850008DF
:101210009D7D0008967D000862890008887D000891
:101220000022002904D003789A18401C491EF8E7D0
:10123000D0B27047FEB50293009201910446089F18
:10124000B81D2070661C0120020200253046294688
:1012500003F090FF27710098E0700198A070AA2019
:101260006070601D02993A4603F06CFF2078871E7B
:1012700030463946FFF7D4FFF05520788019401EDC
:10128000552101702846FEBDF8B50746002500919E
:10129000A94214D0785DAA280FD17E19F4783019AC
:1012A0004079552809D1211D3046FFF7B9FF39197A
:1012B00049190979814200990AD06D1CE8E7032099
:1012C000124901221EA306F04BFB00252846F8BD5B
:1012D000E01C03F043FE002813D005467078287008
:1012E000B078AC706870002C04D0311DE81C224628
:1012F00003F028FF07200549012205A306F030FB73
:10130000E4E703200149012208A3DCE77085000817
:1013100048525F476574446174614672616D65202F
:101320005375636365737321000000006765742063
:101330007370616365206661696C0D0A00000000CE
:1013400048525F476574446174614672616D6520FF
:101350004661696C21000000F0B5DFB005460EA8BB
:101360004021FEF77CFF6C782D78082C22D8A00055
:1013700001A108588746C0469D130008B91300080C
:10138000E5130008F91300080D14000821140008E3
:101390003514000883140008B514000807268B498B
:1013A0000122A14B304606F0DBFA0EA8FFF72AFC1B
:1013B00000254CE000264AE00095072683490127D6
:1013C000984B30463A4606F0CBFA0EA938460F46FF
:1013D00029463A46FFF7BCFB002838D03878002869
:1013E00061D034E000950726784901228C4B3046C5
:1013F00006F0B6FA022026E000950726734901227E
:10140000864B304606F0ACFA03201CE00095072618
:101410006E490122804B304606F0A2FA042012E009
:10142000009507266949012275A3304606F098FA0F
:10143000052008E000950726644901226BA3304689
:1014400006F08EFA06200EAA2946FFF781FB601EE1
:10145000C0B2052806D8002D04D10EA800213246BE
:1014600003F088FE00961EAE0EAB3046294622469B
:10147000FFF7E0FE3178701C00F0A8F900205FB0A3
:10148000F0BD009507265149012751A330463A4641
:1014900006F066FA0EAA30463946FFF759FB0028D7
:1014A000D5D0002D5ED00EA800210726324603F0CD
:1014B00061FECCE71EAF00200B90B87038800DAEF7
:1014C0000C96B070308030463946FFF7A5F9717838
:1014D0000F220B0911400A26734358180A900EA9CF
:1014E00088700C988378180913407043C0180990CD
:1014F000C8703878030910407343181808900871B1
:1015000078780309104073431B184B71B8780709AA
:1015100010407743381888710C9F3F783A403F0954
:101520007743BA18D6B2303A4A707D221201B21807
:10153000160A0E70C1B2DBB20898C6B20998C7B2DB
:101540000A98C0B200920190029703960493059105
:101550000AA006900BA11AA21BA30B9800F0AAFAEE
:10156000072674E70EA84078002802D00EA807705E
:101570001EE70EA800250726294697E71B5B306D5E
:10158000000000002020257325736B4765744375A8
:101590007272656E7454696D653A20253034642D1D
:1015A000253032642D253032642020253032643AD3
:1015B000253032643A253032640D0A25730000006C
:1015C0001B5B313B33326D00493A200070850008C7
:1015D0006B53656E736F724661696C7572655265A7
:1015E000636F726428256429000000006B506F77D8
:1015F00065724F6E5265636F72642825642900001E
:101600006B506F7765724661696C75726552656380
:101610006F72642825642900528500082D85000812
:101620003E8500081C850008778500088AB002A85E
:101630002021FEF714FE204C214D204E2068002171
:10164000C94304F04BFA0724012201922046314697
:101650002B4606F085F91B4D284602F0A2FBC7B2C7
:10166000009720463146019A17A306F079F902AC9B
:101670002846134D21463A4602F0B6FB102116A02B
:1016800022460D4C3B4606F04BF8062FD6D302A857
:101690003946FFF7F9FD0746002808D0BB78FA1C49
:1016A000102111A006F03CF83846FFF755FE3846E9
:1016B00003F0DEF9C2E7C046A008002070850008EC
:1016C000668500087C0100206275665F6C656E208F
:1016D0003D2025640A0000006C7075617274315FF2
:1016E00072785F7262000000486F73744672616DB9
:1016F00065446174610000007CB503F085FB01A8BE
:10170000002101703D4E306880060AD5F0698006E0
:1017100007D5706A01A908705C484C30012202F0BC
:10172000E0FB3068000616D5F069000613D5574C6B
:101730006034204602F035FB002808D001AD0122BC
:101740002046294602F050FB2878B06203E030685A
:101750008021884330603068400607D5F069400634
:1017600004D5402030623168814331603068C00761
:1017700007D0F069000704D540203062706A01A9E3
:10178000087003F05BFB7CBD70B50C4605463F4E10
:1017900030464C3031461431102202F016FB6036D0
:1017A00008498022304602F010FB00F029F8284654
:1017B000214600F023FD062035490122024B06F0A8
:1017C000CFF870BDD80F00201E95000870B50C46EC
:1017D00005462E4E6036304602F0CEFAA04201D2C7
:1017E000002070BD30462946224602F07AFB0349AC
:1017F0000A68802313430B6070BDC0460080004020
:10180000F0B587B01148016802263143016000BF7E
:1018100000BF00BF00200190059003960127F80249
:101820000290062406940497094802AD294605F063
:101830009BFB019805900396B802029006940497CA
:101840000348294605F090FB07B0F0BD2C1002407C
:1018500000040050BCB50D4D28464C3002F0A1FAF2
:10186000044600280ED02868A0420BD1009407201F
:101870000749012207A306F073F80B48006804F03B
:10188000E9F801E0002C00D02C60BCBD3001002044
:101890002A9500086C7075617274315F72785F729E
:1018A000623A202564000000A00800200120000208
:1018B00002490A6802430A607047C0461810024095
:1018C00010B508300F24044008012018C0B21F21B1
:1018D0001140DA06920D5118029A9206120C8918DC
:1018E00009020C18204600F037FA0006201810BD37
:1018F00080B503F089FA15484168890404D5016C64
:10190000890701D50221816411490A68D20704D0F0
:101910008A68D20701D001220A614168C90404D54E
:10192000016CC90701D0012181640168490709D50B
:10193000016C490306D50121890481640549C81C4D
:10194000FEF76AFF03F07AFA80BDC0461428004013
:101950002CB0004090000020BCB5002401AD012255
:101960002046294600F00AF8012801D0E043BCBD1A
:101970002878BCBD80B500F005FC80BD10B50B46D5
:10198000EFF31084012181F31088194600F004F868
:1019900084F3108810BD0000FEB50B460546444C8C
:1019A0002078532805D01E46174600F0EBFB3A4638
:1019B0003346182068432418E76E266FBE4217D9B5
:1019C000606E0292A26E8119951B0298854200D327
:1019D0000546019318462A46FEF728FC029AAE19DE
:1019E000A06E864200D10026521B019B5B1900E0CD
:1019F0000025BF1B974200D31746002F07D0606E0B
:101A0000811918463A46FEF711FCBE197D19002DC2
:101A100001D0703426602846FEBDC046F8B5144695
:101A20000D46064622480078532801D000F0AAFB54
:101A3000EFF31087012181F31088304629462246B2
:101A400000F004F887F31088F8BDC046F8B51446D6
:101A50000D461821414316484618F06A18360228E8
:101A600010D0012815D0002700281ED1304600F0E4
:101A7000B9FBA04219D330462946224600F0A2FD08
:101A8000274612E030462946224600F06DFD074603
:101A90000BE0304600F0A6FB0746A04200D32746E5
:101AA000304629463A4600F08DFD3846F8BDC0461E
:101AB000E001002082B0E0B50492059304AA0192EF
:101AC00001AA00F005F88CBC02BC02B00847000077
:101AD000F0B59FB007920E4602901E9000271C970B
:101AE00040201B900AA81A901D9731783046761C2A
:101AF000252906D0002900D11AE11AA800F03EFCE1
:101B000090E0801C00253178232907D02B2907D0AD
:101B10002D2907D030290AD1022104E0082102E052
:101B2000042100E001210D43401C761CEBE700245A
:101B30000897302909D3392917D80A226243541843
:101B4000303C401C7178761CF3E72E290DD100271C
:101B50000921CA4301780B463A3B934207D30A2234
:101B60007A435718303F401CF2E7002700E0064652
:101B7000761C0846633809280DD8C0467844007999
:101B800040008744545A4F4F4F044F4F4F04701C2E
:101B900031780646EDE708467038082815D8C04663
:101BA0007844007940008744043D3D1E3D313D3D71
:101BB0001400079A1068011D1160016800200823B5
:101BC000009301901AA810222AE0252958D05829FC
:101BD00028D1079A1068011D1160016800940195D1
:101BE0001AA810221BE0079A1068011D11600468F2
:101BF000002C00D156A42178002913D01AA800F097
:101C0000BDFB641C1D980028F5D50BE0079A1068F1
:101C1000011D11600168009401951AA80A223B4633
:101C200000F02AFB1D9F002F00D45EE78DE0079A8D
:101C30001068011D116001785FE7079A1068011DA7
:101C400011600268D01711464140081A06925142AD
:101C50000491012109910A2805D30A21FEF75CFBB2
:101C60000999491CF6E70998B84200D80997002C51
:101C700009D00698002801D4680705D5641E03E042
:101C80001AA825213AE7002402212940059603914C
:101C900001D0002F13D0E80711D1002C0FD0661E01
:101CA000A6420CD20998A04209D21AA8202100F01D
:101CB00065FB1D98089000283446F0D521E008986F
:101CC0000028059EAED40698002804D4680704D4E2
:101CD000069804900AE02D2102E02B21069804903A
:101CE0001AA800F04BFB1D9800289BD403980028ED
:101CF00009D1009401951AA80A2204993B4600F0E4
:101D0000BBFA059E8EE7012028403843F1D1002C14
:101D1000EFD0661EA642ECD20998A042E9D21AA8DA
:101D2000302100F02BFB1D9800283446F1D5E8E760
:101D3000002F09D01C9D002D04D00AA902982A4624
:101D4000FFF76CFEEF1900E0002738461FB0F0BD2A
:101D5000284E554C4C2900000F2101400206120F5D
:101D60005118C204D20E89188203D20E89180002BB
:101D7000800E0818704780B503F046F804F05CFC4C
:101D800003F05CF880BD000010B51D4CA068800613
:101D9000400F411E032922D81A48C04679440979C8
:101DA00049008F4421011619E168C90700D11E4876
:101DB000E1680906C90E00D120214843E1684905C0
:101DC000490F00D10821FEF7A7FAE1684903890FFE
:101DD00009E07D20000207E00120C00304E0206844
:101DE000C004810F1048C840A16889091C220A401C
:101DF00005498958FEF790FA0A49086010BDC046A7
:101E00000010024000127A00687D0008034804496F
:101E100001600448044901607047C04608ED00E0D5
:101E2000000000080C0000200024F40000F0E6FB95
:101E3000BCB50C460021019103280CD16068FEF767
:101E400049FA0546A068FEF745FA0246E9B201A83C
:101E5000FEF704FFBCBD03200249012202A305F0E6
:101E60007FFDBCBD91850008544553545F466C61AD
:101E700073685F526561645F5265636F72642020AE
:101E8000202020202D2D757365205F636D645F20F9
:101E90005B7265636F726428307E36295D205B6EED
:101EA000756D5D00FEB503281FD10C464868FEF72E
:101EB00011FA0546A068FEF70DFA0446EDB20126B8
:101EC0002A4FA64217DC009501961C48029000207C
:101ED0001BA1244A244BFFF7EDFD2846FFF770F8BD
:101EE000384604F003FA761CEBE70320024901228E
:101EF00002A305F035FDFEBD9185000854455354FD
:101F00005F466C6173685F57726974655F526563A1
:101F10006F72642020202020202D2D757365205F96
:101F2000636D645F205B7265636F726428307E3618
:101F3000295D205B6E756D5D00000000A3850008C3
:101F4000202025732573466C6173685F577269742E
:101F5000655F282564295265636F72643A25640DB4
:101F60000A257300B08500088D85000860EA00002E
:101F7000F8B50C460546804F384624300C4980227F
:101F800001F023FF3837012672020A49384601F072
:101F90001CFF00F039F800F093F82846214600F0C5
:101FA000A1FA06206D49044B324605F0D9FCF8BD74
:101FB0008C130020841C00201E95000880B502F0C0
:101FC00023FF10480168C90504D5C169C90701D0BC
:101FD000012101620168C90704D0C169C90701D0A4
:101FE000012101620168C90608D5C169C90605D584
:101FF00010210162F548406803F02CFD02F01EFF3D
:1020000080BDC04600380140F0B587B02248016865
:1020100001252943016000BF00BF00BF06270297CA
:1020200000260096E802069005961020049003967C
:1020300001966C46204604F007FF0297009506962D
:1020400005960496202003900196204604F0FCFE9D
:10205000124C2068022101432160206804210143C1
:1020600021602068082101432160FF2001020C4A01
:1020700013688B43136069027E4B1960000411687A
:1020800081431160A80218603D4800F00BF82068F9
:102090002843206007B0F0BD301002400800024025
:1020A00008E400E0F8B58021039102900348019014
:1020B00000200090684604F0E5FE8FBD2438014002
:1020C000F0B587B01248016801263143016000BFB6
:1020D00000BF00BF00200190059002270397F00287
:1020E0000290069604960520040702AD2046294674
:1020F00004F03AFF0198059003973003029006968A
:1021000004962046294604F02FFF07B0F0BDC046D4
:102110002C10024007201149012211A305F020FCD8
:10212000D04E164F70680021C94303F0D7FC3C68BD
:1021300080210D1B32699542F4D0114880189542D8
:1021400001D9A91A06E0891A00F038F9802C03D0C9
:102150000B48294600F032F93561E3E72A9500087B
:1021600055617274315F52785F5468726561645F63
:10217000456E747279000000300100200C000240AE
:10218000EC06002010B5124CA8212046FEF767F897
:102190000320206160610F49A1610F48E0610120C7
:1021A000800220620020A0626062E06221660B492A
:1021B00061661021A1662067E066606708490F31FB
:1021C000102804D00A782254491E401CF8E710BD9C
:1021D000E0010020339500089C0200208C020020C2
:1021E000C07B0008C2680169914201D9D04302E076
:1021F000D2438918806808187047000070B588B00D
:102200000022079203239B02174CA6689E430125D8
:10221000EB02F318A3602B0526681E43266000BF5F
:1022200000BF00BF069103900192059204920C201A
:1022300002900E4C01A9204604F0E3FE002800D0D5
:10224000FEE70B48016840220A43BF218A4302602F
:102250002807C449086020682021014321602068C4
:102260002843206008B070BD341002400080004058
:102270001CE400E000E100E0F0B587B003931746EE
:10228000059001260D9D0C9C01910846B84204D38F
:102290003946FEF741F8761CF8E706970127039BBD
:1022A0009E4200D81E4628463840002C04960290D4
:1022B00018D0002816D12020A90701D4054600E037
:1022C0003025002B00D00546002C0BD0A64209D2A9
:1022D000059E3046294600F051F8641EF068049EC1
:1022E0000028F1D50598C06800283DD40094019DD0
:1022F000039C022C02D3641E069906E02846394648
:10230000FEF70AF80699884201D34F43F1E7059E8C
:1023100028463946FEF700F8044614A0015D304611
:1023200000F02CF8F068002809D47C432D1B3846B7
:10233000069C2146FDF7F0FFA7420746E8D2029827
:102340000028049E00980FD000280DD0059D441E43
:10235000844209D2864207D22021284600F00EF896
:10236000E86800282046F2D507B0F0BD303132339E
:1023700034353637383941424344454610B5044672
:1023800042688368581C904201D9184606E02268CA
:10239000D154A060E168491CE1606268904208D1B4
:1023A00021682069FFF73AFBA168884202D100202A
:1023B000A06010BD0020C043E06010BD80B50A469B
:1023C00001462848243001F08CFD80BD30010020FA
:1023D0001FB51FA00021012203F0E4FA214C606028
:1023E000002807D120480090002020A12BA22DA377
:1023F000FFF760FB022000902BA02E4900220A2349
:1024000004F0C6F9E060002801D004F055FA052078
:1024100003901420029028480090FD20C0000190F5
:10242000264827A12A4A002303F022FF00280BD1C7
:10243000224803F0DFFF0C4900900191002025495C
:1024400025A227A3FFF736FB002004B010BDC0462D
:1024500075617274315F72785F636865636B5F7317
:10246000656D000030010020A38500082020257341
:1024700025736372656174652075617274315F7272
:10248000785F636865636B5F73656D206372656118
:102490007465206661696C0D0A2573001B5B313B16
:1024A00033306D00443A20006C7072785F74696D4F
:1024B00065000000551800089C1400200C14002032
:1024C00075617274315F72785F74687265616400FF
:1024D00015210008EC9400081B5B313B33326D0082
:1024E000493A2000B0B588B00125AA031A4B1C68F0
:1024F00014431C6000BF00BF00BF0022079206917A
:102500000592049203900C2001900292134C01A9B1
:10251000204604F031FF002800D0FEE7FF20000233
:102520000F490A6882430A6068060E49086028025B
:102530002168014321602068284320602068102121
:1025400001432160A06840210143A1602068284325
:10255000206008B0B0BDC0463810024000380140CD
:1025600018E400E000E100E0FEB516460D46C7683D
:10257000002101900269BA42029103D9F94354182B
:10258000816803E0F9435218816854184268C91BF6
:102590008C4200D30C46B44200D33446D0192946AD
:1025A0002246FDF743FEE719019881688F4200D16A
:1025B00000270299C760361B2D196118002ED9D14A
:1025C0000846FEBDF8B5154604464068A268E668B0
:1025D0008019971BBD4204D22A46FDF727FE7519C4
:1025E00009E00E463A46FDF721FEF119ED1B606841
:1025F0002A46FDF71BFEE560F8BD0000BFF34F8FD4
:10260000034804490160BFF34F8F00BFFDE7C04698
:102610000CED00E00400FA0580B5012000F0F8FDA3
:1026200080BD7047002804D0C1B2002903D001202A
:1026300010E000207047FF210A02024002D0110A78
:10264000092007E00904014002D0090C112001E033
:10265000010E1920014A515C40187047D17B0008D7
:10266000FEB5012000F0D4FD0B4F009700240BA114
:10267000124D134E20462A463346FFF71BFA1148E7
:1026800000680090019710A120462A463346FFF7C4
:1026900011FA2046FEBDC046A38500082020257300
:1026A00025735F706572665F636F756E7465725FC8
:1026B000696E69740D0A257300000000B08500087A
:1026C0008D8500080C00002020202573257370657F
:1026D00072665F636F756E74657220696E69742CC3
:1026E0002053797374656D436F7265436C6F636BD0
:1026F0003A25640D0A25730070B515460446002876
:1027000004D1094809A1372201F0B4FF0026002DA9
:1027100006D02A792968A06C03682046984700E013
:10272000F643304670BDC046C69400085F70696EBF
:102730005F636F6E74726F6C00000000B0B586B09E
:1027400014460D4601A81421FDF789FD2806800FC7
:1027500008D1E9B20C20484346490A58521C01D01E
:10276000081800E00020042C15D8C0467C442479C9
:102770006400A744020C10040A00012106E00221B3
:10278000029181680191012104E003210291816895
:10279000019100210391406801A904F0E5FB06B016
:1027A000B0BDC04670B51E4614460546002804D18B
:1027B000084809A1162201F05DFF0020002C08D076
:1027C000082E06D12168A86C82682846904720719F
:1027D000082070BDC69400085F70696E5F72656105
:1027E000640000003F220A400C20504321490A584F
:1027F000521C01D0081800E0002041688068096977
:102800000140091A484248417047C04670B51E460B
:1028100015460446002804D1084809A1262201F0E3
:1028200029FF0020002D08D0082E06D12A7929681A
:10283000A06C436820469847082070BDC6940008E5
:102840005F70696E5F77726974650000002A01D05D
:10285000182000E028203F2211400C224A4305495D
:102860008B585B1C01D0891800E000214A688968F8
:10287000115070471C820008FEB50446089D0646AC
:1028800028362EC61C30E0612062232118462A46D5
:1028900002F070FC234628330FCBD218121F144BC2
:1028A00002F07EFA606225463C350A9E099F202F81
:1028B00004D310A018A1A72201F0DCFE6F70AF7046
:1028C000E664266500202064A063E864286528701B
:1028D0000090019020465430134A2146234603F0CD
:1028E000BFFF12480168002901D020468847FEBD7D
:1028F000256100087072696F72697479203C2052FA
:10290000545F5448524541445F5052494F524954D4
:10291000595F4D41580000005F72745F74687265C2
:1029200061645F696E6974001D650008781100209C
:1029300070B505468826FDF7DDFB0446A959002938
:1029400001D0284688472046FDF7D8FB70BD00001F
:102950000B4A022806D0012809D10320030510687C
:10296000984302E0012041041068084310600120F0
:10297000000411680143116010684003FCD57047E2
:1029800000100240074908684A68801A064A12681F
:10299000520106D50A68121A102A02DB096840188B
:1029A000401C704714E000E004ED00E080B500F04A
:1029B00093FE002080BD80B501F07CF8002080BD32
:1029C000F0B58BB01E460A920D460746109C02F0E9
:1029D0002BFA002809D000960194002039462A4697
:1029E0000A9B04F0A5FD0BB0F0BD0996079535488C
:1029F000016800290A9AF6D0456B002D5ED0234667
:102A0000B800314908180590A620F840012101407E
:102A10000691201F03900894002DE4D02846183812
:102A20000068B84248D32E462C3E281F0468002C6C
:102A30000BD009980090019330463946079A0A9BBB
:102A4000A047089B0A9A002836D028461C38006800
:102A500010430DD02846103804680998009001935F
:102A600030463946079A0A9BA047089B0A9A23E0FA
:102A7000069800281846099C214611D1059800683F
:102A800003F031F9024600280898214608D00F4883
:102A9000049203F028F9049941180398401A611828
:102AA0002A46103A146800910190002330463946B6
:102AB000079AA0470A9A089B2D68ADE7099802F08B
:102AC00025FA90E7841E0020F07C0008639500083A
:102AD00010B5154841692922895C890703D4134838
:102AE000002101701EE00169002905D001200202C9
:102AF0000E48FDF7BFFB15E001F00AFC002803D0EB
:102B00000A480BA1052202E008480BA10722FDF7A5
:102B10008DFB064C2046FDF7BAFB3E2121542018C0
:102B200000214170014810BD980000209C07002042
:102B30006D7368200000000066696E7368200000F5
:102B400010B5074C6069002805D1064806A1C822C7
:102B500001F090FD606902F07DFF002010BDC046CD
:102B600098000020228C000866696E73685F727896
:102B70005F696E6400000000F8B505461C4E706980
:102B8000002804D11B481CA1DB2201F073FD28465C
:102B900001F00AFE00280ED00446852085007069E9
:102BA0004059844206D0FF214431204601F002FE04
:102BB000002805D0F8BD16A0294602F07DF9F8BD21
:102BC00077697859002807D001F0BAFD706940593B
:102BD000002101F0D7FE7769DF204000381854212A
:102BE000FDF73DFB7C510949204601F0CBFEF8BDC5
:102BF00098000020228C000866696E73685F736518
:102C0000745F64657669636500000000412B00080D
:102C100066696E73683A2063616E206E6F74206619
:102C2000696E64206465766963653A2025730A00DD
:102C3000B0B50446094D6869002805D1084809A1C6
:102C4000A72201F017FD68692921425CFD2313408A
:102C5000E207920F9A184254B0BDC0469800002077
:102C6000228C000866696E73685F7365745F7072AA
:102C70006F6D70745F6D6F6465000000FEB5184F76
:102C800018481949396078604320C1000125284659
:102C900001F026FD786100281AD00A201521009144
:102CA0000190AB0211A013490024224603F044F91D
:102CB0000646786910A12246234602F0A7FE284660
:102CC000FFF7B6FF002E08D0304603F093FB04E078
:102CD0000BA002F0F1F80020C4432046FEBDC04620
:102CE000980000206C9700081C96000874736865B3
:102CF0006C6C0000192D00087368727800000000E9
:102D00006E6F206D656D6F727920666F72207368CB
:102D1000656C6C0A000000008AB0614F7869292256
:102D2000815C0123079319430392815485218C0010
:102D30000059002805D101F0FDFC002801D0FFF763
:102D40001BFFFFF7C5FE574802F0B6F800200890B9
:102D5000C543786909A9089A0A70002805D1B322E9
:102D6000554851A101F086FC78690059002810D01F
:102D700009AA0123294601F0B9FD012806D0786986
:102D8000294602F0ABFE78690059F1E709A80678F8
:102D900002E001F06BFF06461B2E04D17869282162
:102DA000079A4254D6E77B692820185CED495A18E7
:102DB00019462831022806D0012821D15B2E1DD1C9
:102DC00002200870C5E7002008703146083905293F
:102DD0005ED93146413903291DD804924900C046C5
:102DE0007944898849008F44030074017B018F0175
:102DF000598D002900D1B0E1481E97E1089808706C
:102E000030460838052806D87844007940008744C1
:102E100080B756090956002E9BD07F2E00D178E04E
:102E2000FF2E96D01088502801D3002010805188A2
:102E3000814200D3FFE0421A5918FF20C030081821
:102E4000DF235B000693C91802F07CF9069B212062
:102E500002017869815A4018C65478690399415C27
:102E6000C90709D0811809884018C118C5A016469D
:102E700002F022F832467869865ABA49415A8E429F
:102E800000D3E6E0B94802F017F8761C7869F4E759
:102E90007944097949008F443C7312111112C046DC
:102EA000980000209C07002066696E73685F676564
:102EB0007463686172000000228C0008B2E79E8D86
:102EC0001088002800D1E2E00492052E059300D27C
:102ED00082E0B72040001818DF214900591850221D
:102EE00002900191FDF7DAF9059B002800D1CEE0B0
:102EF0001E467E360420002800D1BAE006903046F7
:102F0000503850223146FDF791F90698401E503650
:102F1000F1E75188002900D11BE7481E5080164672
:102F20001288521E328080B292B2824277D9121A2F
:102F300006921A46DF235E00931918185918069A4C
:102F400002F000F978698749415A401800218155FB
:102F50002120010106917869415A4018811986A003
:102F600001F0AAFF78690699465A7E49405A86427E
:102F700000D9EEE67D4801F09FFF761C7869F4E702
:102F8000089E21200001185A864205D2774801F098
:102F900093FF761C7B69F4E775481E4601F08CFFB1
:102FA000DF2040000690361801F0B2F9012802D166
:102FB000304601F031F8FFF78BFD71486849324621
:102FC00001F07AFF7E6906983018FDF760F96549CF
:102FD000705271184880BCE6002E0CD0DF204000F3
:102FE0001918502210467043C0182238FDF756F9C0
:102FF000059B00284BD050214E439E192E3630465B
:10300000FDF72DF9DF204000059909180498028882
:103010003046FDF70BF9059B988D461C36E055A010
:1030200001F04AFF78694F49415A4018DF214900B1
:10303000002242548DE61818DF2149004654786971
:103040000399415CC90704D04748314601F034FF79
:103050007869444A815A491C815280184288521C1E
:10306000428089B2502900D273E60021418001805C
:103070006FE65021029E3046FDF7F1F80498028871
:1030800030460199FDF7D2F8059B05269E855E85A1
:1030900001F03EF901280FD178690399415CC90715
:1030A00003D0334801F008FF78692E49415ADF22E6
:1030B0005200801801F008F8FFF70AFD284801F0D7
:1030C000FBFEDF204000796908185421FDF7C7F89E
:1030D0003FE6598D9A8D501E884224DD481C25E01C
:1030E000049E70883188884200D332E61818DF21A8
:1030F0004900415C1C4801F0DFFE21200001796994
:103100000A5A521C0A5224E604984088002800D12A
:103110001FE6164801F0D0FE2120000179690A5A05
:10312000521E0A5215E6002A00D112E65885DF2108
:1031300049005E1880B25022504319182E31304693
:103140000593FDF773F83046FDF7A1F8049E7080F3
:103150003080059803F028FEFBE55885F9E5C04668
:103160009C0700200E020000338C0008208C000811
:10317000AD8C0008082008000825732020080000F6
:10318000368C00082573000010B5064C01F04CFE8B
:10319000002803D005208001241800E038342046A0
:1031A00010BDC046841E002070B5EFF31084EFF30D
:1031B000108072B600252A4E28462946002D15D1CA
:1031C000FFF7E0FBC217716A336A18185141F26ABF
:1031D000B36AC31A0B46934102DAF16AB06A01E09E
:1031E000B062F16284F310882D1FE7E770BDC0461E
:1031F00080B502A001F060FE002080BD48656C6CC7
:103200006F2052542D546872656164210A000000D9
:1032100070B5EFF31081EFF3108272B600220F4BFE
:10322000114C104D002A0ED1002805D100261E6039
:103230005D609E6007261E6001267606266081F38B
:103240001088121FEEE704F035FC054800214162AA
:10325000016281600161FFF7E4F970BD10E000E0F8
:10326000B0010020FFFFFF0004ED00E0F8B50EA064
:1032700001F022FE114805681148076811A4AF4209
:1032800010D23E68022230462146FDF714F800288D
:1032900006D07A680CA0314601F00EFE074805689A
:1032A0000C37ECE70020F8BD2D2D46756E63746970
:1032B0006F6E204C6973743A0A0000009C00002075
:1032C000980000205F5F0000252D313673202D2DE2
:1032D0002025730A00000000F0B593B009242046B1
:1032E00002F0E4F90EA90C72002412940821119145
:1032F00006A90F91001D0E901FA0102128A201F019
:10330000DBFD01F007F828A001F0D6FD029420466D
:103310000EAE314600F006F90390307A049006AF05
:1033200012980590029D059885421FDA3E68341F69
:10333000FCF7E0FE21787F220A4004998A4210D1EE
:10334000FCF7DCFE307AB17B019180001F49085800
:103350000090143E10211EA00A46334601F0ACFD39
:1033600001E0FCF7CBFE3F1D6D1CDCE70398002855
:10337000CED1002013B0F0BD252D2A2E73202020A1
:1033800020202020202074797065202020202020FB
:1033900020202072656620636F756E740A0000003D
:1033A0006465766963650000202D2D2D2D2D2D2D52
:1033B0002D2D2D2D2D2D2D2D2D2D2D2D2D202D2D4A
:1033C0002D2D2D2D2D2D2D2D0A000000107D0008F6
:1033D000252D2A2E2A7320252D32307320252D38B5
:1033E000640A0000F0B595B00424204602F05EF9AE
:1033F00010A90C72002414940821139108A91191AA
:10340000001D109028A0102130A201F055FD00F001
:1034100081FF30A001F050FD0394204610AC2146FE
:1034200000F080F80490207A069008AE1498079077
:10343000039D0798854230DA3468271FFCF75AFE4F
:103440003F78FCF75BFE7F2038400699884221D107
:103450002746143F2169A0680834A04213D02046B3
:10346000059101F071FD059900910190102121A0B5
:103470000A463B4601F020FD204603F0ADFC234800
:1034800001F01AFD06E00091102121A00A463B46FA
:1034900001F012FD361D6D1CCBE704980028BDD14C
:1034A000002015B0F0BDC046252D2A2E7320202007
:1034B0002020207365742020202073757370656E42
:1034C00064207468726561640A0000006576656E48
:1034D0007400000020202D2D2D2D2D2D2D2D2D2D76
:1034E000202D2D2D2D2D2D2D2D2D2D2D2D2D2D0A3C
:1034F00000000000252D2A2E2A7320203078253048
:10350000387820253033643A00000000AD8C000884
:10351000252D2A2E2A732020307825303878203027
:103520000A000000F8B5064600250D61C8680028AD
:1035300028D00C46087A002824D000952768002E51
:103540003D4600D03546FCF7D5FD002E06D0311F94
:1035500009787F220A40217A8A4210D162680021CC
:103560000E462D68BD4205D020C2761CE3689E42FF
:10357000F7D100E00D46FCF7C1FD266102E0FCF743
:10358000BDFD009D2846F8BDF0B597B00524204646
:1035900002F08CF812A90C720024169408211591DF
:1035A0000AA91391001D12902CA0102134A201F041
:1035B00083FC00F0AFFE34A001F07EFC03942046B3
:1035C00012AC2146FFF7AEFF0490267A0AAD16989A
:1035D0000890039905960898814239DA09912C6878
:1035E000271FFCF787FD3F78FCF788FD7F203840D8
:1035F000B04229D107952746143FA58AE08A069054
:10360000A6680834204601F09FFCA64210D0069917
:10361000009101950290102122A00A463B4601F03C
:103620004BFC204603F0D8FB244801F045FC09E0A0
:103630000699009101950290102121A00A463B466F
:1036400001F03AFC059E079D2D1D0999491CC2E712
:1036500004980028B4D1002017B0F0BD252D2A2EE3
:103660007320656E7472792073697A65207375733F
:1036700070656E64207468726561640A0000000001
:103680006D61696C626F7800202D2D2D2D20202D0D
:103690002D2D2D202D2D2D2D2D2D2D2D2D2D2D2D67
:1036A0002D2D0A00252D2A2E2A7320253034642042
:1036B00020253034642025643A000000AD8C0008D9
:1036C000252D2A2E2A7320253034642020253034DD
:1036D000642025640A000000B0B5064DA96806A064
:1036E0000A4CA047A9690AA0A047E9690DA0A04714
:1036F000B0BDC046BC000020746F74616C206D6565
:103700006D6F72793A2025640A000000B94E0008F6
:1037100075736564206D656D6F7279203A2025643C
:103720000A0000006D6178696D756D20616C6C6FC9
:103730006361746564206D656D6F72793A202564EC
:103740000A000000F0B595B00624204601F0AEFF57
:1037500010A90C72002414940821139108A9119146
:10376000001D109029A010212FA201F0A5FB00F050
:10377000D1FD30A001F0A0FB0294204610AC214600
:10378000FFF7D0FE0390267A08AD149806900299B0
:1037900004960698814233DA07912C68271FFCF7BC
:1037A000A9FC3F78FCF7AAFC7F203840B04223D127
:1037B00005952746143F258BA6680834204601F05E
:1037C000C3FBA6420ED00095019010211FA00A460F
:1037D0003B4601F071FB204603F0FEFA204801F061
:1037E0006BFB07E00095019010211EA00A463B46A6
:1037F00001F062FB049E059D2D1D0799491CC8E739
:1038000003980028BAD1002015B0F0BD252D2A2E2E
:103810007320656E7472792073757370656E6420A1
:103820007468726561640A006D73677175657565AA
:1038300000000000202D2D2D2D20202D2D2D2D2D93
:103840002D2D2D2D2D2D2D2D2D0A0000252D2A2E2F
:103850002A732025303464202025643A00000000BB
:10386000AD8C0008252D2A2E2A73202530346420A3
:103870002025640A00000000F0B597B0032420461C
:1038800001F014FF12A90C7200241694082115915E
:103890000AA91391001D129022A010212AA20691BC
:1038A00001F00AFB00F036FD29A001F005FB0494AD
:1038B000204612AF3946FFF735FE0590387A08905A
:1038C0000AAD16980990049E0998864224DA2F685A
:1038D0003C1FFCF70FFC21787F220A4008998A429E
:1038E00015D1FCF70BFC7C69F87C07903846083052
:1038F00001F02AFB069900910194079A0292039025
:10390000143F1BA00A463B4601F0D6FA01E0FCF743
:10391000F5FB2D1D761CD7E705980028C9D100209E
:1039200017B0F0BD252D2A2E732020206F776E65ED
:10393000722020686F6C642073757370656E6420EC
:103940007468726561640A006D75746578000000C2
:10395000202D2D2D2D2D2D2D2D202D2D2D2D202DBE
:103960002D2D2D2D2D2D2D2D2D2D2D2D2D0A000004
:10397000252D2A2E2A7320252D382E2A7320253016
:1039800034642025640A0000F0B595B00224204676
:1039900001F08CFE10A90C720024149408211391DC
:1039A00008A91191001D109029A010212FA201F04B
:1039B00083FA00F0AFFC30A001F07EFA02942046BA
:1039C00010AC2146FFF7AEFD0390267A08AD14989F
:1039D0000690029904960698814233DA07912C6882
:1039E000271FFCF787FB3F78FCF788FB7F203840D8
:1039F000B04223D105952746143F258AA66808348E
:103A0000204601F0A1FAA6420ED0009501901021A7
:103A10001FA00A463B4601F04FFA204603F0DCF9AE
:103A20001F4801F049FA07E00095019010211DA000
:103A30000A463B4601F040FA049E059D2D1D07995C
:103A4000491CC8E703980028BAD1002015B0F0BD82
:103A5000252D2A2E73207620202073757370656EB5
:103A600064207468726561640A00000073656D61AA
:103A700070686F7265000000202D2D2D202D2D2DDA
:103A80002D2D2D2D2D2D2D2D2D2D2D0A000000003D
:103A9000252D2A2E2A7320253033642025643A00F0
:103AA000AD8C0008252D2A2E2A7320253033642062
:103AB00025640A00F0B593B00124204601F0F6FD1C
:103AC0000EA90C72002412940821119106A90F91DD
:103AD000001D0E903048102130A201F0EDF900F0E9
:103AE00019FC30A001F0E8F9029420460EAF3946E7
:103AF000FFF718FD03903F7A12980590029D0497F6
:103B00000598854241DAA80006A90E58341FFCF733
:103B1000F1FA21787F220A40BA4232D13446283461
:103B2000FCF7ECFA607800903346143B10212DA08E
:103B30000A4601F0C1F921780F200840042804D872
:103B400080002BA1085801F0B7F9F4690020215C2E
:103B5000401C2329FBD0376A391A6420484364305B
:103B60003946FCF7D9FB03463069F16B726A009164
:103B700001923919091A23A03A4601F09DF9049FD0
:103B800001E0FCF7BBFA6D1CBAE703980028ADD141
:103B9000002013B0F0BDC046978A000874687265B3
:103BA00061640000202D2D2D20202D2D2D2D2D2D5B
:103BB0002D202D2D2D2D2D2D2D2D2D2D202D2D2D4F
:103BC0002D2D2D2D2D2D2D20202D2D2D2D2D2D204C
:103BD000202D2D2D2D2D2D2D2D2D2D202D2D2D0A52
:103BE00000000000252D2A2E2A7320253364200092
:103BF000DB8A0008ED8A0008FA8A0008E28B0008D8
:103C0000E48A000820307825303878203078253054
:103C100038782020202025303264252520202030AF
:103C2000782530387820253033640A00F0B593B019
:103C30000A24204601F03AFD0EA90C7200241294C9
:103C40000821119106A90F91001D0E9025A01021A9
:103C50002EA201F031F900F05DFB2EA001F02CF94D
:103C6000029420460EAF3946FFF75CFC0390387A89
:103C7000049006AD12980590029C0598844225DABE
:103C80002F683E1FFCF736FA31787F220A400499EC
:103C90008A4212D1FCF732FAB869F96900900191B1
:103CA0003B46143B10212AA00A4601F005F9F81EF4
:103CB0000078C00704D12F4803E0FCF71FFA02E0A8
:103CC00029A001F0F9F82D1D641CD6E703980028FF
:103CD000C8D102F0ADFC014617A001F0EDF80020BC
:103CE00013B0F0BD252D2A2E732020706572696FE8
:103CF00064696320202074696D656F7574202020CD
:103D000020202020666C61670A00000074696D65E0
:103D100072000000202D2D2D2D2D2D2D2D2D2D202F
:103D20002D2D2D2D2D2D2D2D2D2D202D2D2D2D2DD0
:103D30002D2D2D2D2D2D0A0063757272656E742048
:103D40007469636B3A3078253038780A00000000D7
:103D5000252D2A2E2A732030782530387820307887
:103D600025303878200000006163746976617465DD
:103D7000640A00008A8A00080146002000290FD04A
:103D80000A68002A0CD04A68002A09D08868C968E5
:103D9000884204D001D9421A01E0511A0A18501E73
:103DA00070470146002000290ED00A68002A0BD077
:103DB0004A68002A08D08B68C968994204D001D9A2
:103DC000C81A70478818C01A704703460020002B95
:103DD00009D0002907D0002A05D0002006C31860AA
:103DE0005860986001207047E0B50023019300936C
:103DF00001AB00F004F8002800D001988CBDF0B5AC
:103E000085B00026002845D005460768002F41D020
:103E1000686800283ED000293CD01446002A39D0DA
:103E200002AA0BC22846FFF7BCFF002832D0A042EE
:103E300002D20A99C9072DD1A04200D32046AA6810
:103E400002998E1A864200D306460446B918039F8B
:103E5000384601923246FCF7E9F90294A41B05D0DA
:103E6000B81929682246FCF7E1F901E001983418F5
:103E70006868844200D30024AC602B69002B03D017
:103E800000212846029A984701260498002801D06C
:103E900002990160304605B0F0BDF8B50024002855
:103EA0001DD005460068002819D06F68002F16D075
:103EB0000E46002913D02846FFF773FF0446B04290
:103EC00000D33446A8680019C11B00D30846A86077
:103ED0002B69002B03D00021284622469847204614
:103EE000F8BDE0B500230193009301AB00F004F8A6
:103EF000002800D001988CBDF0B585B000260028C0
:103F000046D005460768002F42D0686800283FD099
:103F100000293DD01446002A3AD002AA0BC22846F6
:103F2000FFF72AFF002833D00146A04202D20A98A8
:103F3000C0072DD1A14200D32146EA680298861A13
:103F40008E4200D30E46B8180C46039F39460192A4
:103F50003246FCF76BF90294A41B05D0B919286806
:103F60002246FCF763F901E001983418686884423E
:103F700000D30024EC602B69002B03D001212846DC
:103F8000029A984701260498002801D002990160FE
:103F9000304605B0F0BD000082B018240025204650
:103FA000294601F01FFC0DA0009401900DA114A260
:103FB00015A32846FDF77EFD7D20C40018250121AC
:103FC000284601F02DFC204602F090F900212846F9
:103FD00001F026FC204602F089F9EFE71B5B306D0B
:103FE000000000002020257325734C4544305F50AD
:103FF000494E203D2025640D0A0D0A25730000005E
:104000001B5B313B33306D00443A200080B500F03B
:1040100083FBFFF7C1FF80BDFEB504460078002892
:1040200047D0254800680290244806680027019779
:1040300000940298864234D23568062228462049E8
:10404000FCF739F900282AD12046FCF720F902466E
:10405000AD1D20462946FCF72EF900281FD10198F6
:10406000002803D12846FCF712F92F4601900024BE
:10407000385D002806D0295D002903D0884201D18F
:10408000641CF5E70FA0294600F016FF0198844252
:1040900000DB04460848006802900194009C0C363E
:1040A000C7E7002F04D020463946019A01F035FEBB
:1040B000FEBD00F0EFF8FEBD9C000020980000203F
:1040C000198C000825730A00F0B58BB00D46044624
:1040D000002D07D02078202801D0092804D16D1E9A
:1040E000641CF5E70020ADE00021C0B2092808D02B
:1040F000202806D08D4203D060184078491CF4E790
:1041000029460191002900D18DE00198801D009081
:104110004D48006802904D4806680298864200D3D8
:1041200081E03768062238464949FCF7C4F8002880
:104130000AD1B81D2146019AFCF7BDF8002803D129
:104140000098385C002801D00C36E6E7B068029091
:10415000002868D003A82021FCF781F8002220461F
:104160001646AA4258D20378202B01D0092B08D139
:10417000AA4204D200210170521C401CF3E72946D8
:1041800000E01146082E35D2A94245D2B200222BBA
:1041900013D1401C03AB985003784A1C222B1AD031
:1041A000AA4218D25C2B05D14378222B02D1401CA5
:1041B000891C00E01146401CEEE703AB9850771CC9
:1041C0000023C65CCA18092E0DD0202E0BD0AA429F
:1041D0000ED25B1CF5E7761CAA421FD200220270A9
:1041E0008A1C401CBDE7C018AA423E46B9D315E060
:1041F0003E4613E017A000F05FFE03AF1DA5019639
:10420000002E05D002CF284600F056FE761EF7E7B6
:10421000194800F051FE019E002E04D003A930463B
:10422000029A90470EE02046017820220A43202A75
:1042300001D0401CF8E70025057010A0214600F0D1
:104240003BFEE8430BB0F0BD9C000020980000202E
:10425000198C0008546F6F206D616E792061726750
:10426000732021205765206F6E6C79205573653A55
:104270000A00000025732000AD8C000825733A2049
:10428000636F6D6D616E64206E6F7420666F756E06
:10429000642E0A00F8B510A000F00EFE154805685F
:1042A00015480768164CAF4210D23E6806223046C9
:1042B0002146FCF700F8002806D17A68B11D11A04C
:1042C00000F0FAFD0B4805680C37ECE70B4800F0EE
:1042D000F3FD0020F8BDC04652542D54687265614C
:1042E00064207368656C6C20636F6D6D616E6473C0
:1042F0003A0A00009C00002098000020AD8C0008C5
:10430000198C0008252D313673202D2025730A00C5
:1043100001207047B0B50F20C54304A4002D04D080
:10432000204600F0C9FD6D1CF8E7B0BD2D0000006F
:10433000B0B5184C6068002808D000F075FD002862
:1043400005D04F208500FBF7D5FE6051B0BD02F0CF
:1043500017F80028F5D008340020C143204600F0AB
:10436000EFFFB0BD10B50B4C6068002808D000F01E
:104370005BFD002805D04F2080002058FBF7BEFED3
:1043800010BD01F0FDFF0028F5D00834204600F0F4
:104390003DFF10BD841E002070B504461F4DE86827
:1043A000A04204D91EA02649A12200F063F9286981
:1043B000A04204D823A02249A22200F05BF9608821
:1043C000002804D02AA01E49A32200F053F96168F6
:1043D000E8684218A2420FD05388002B0CD12B69F9
:1043E0009A4209D06969914200D16C61516861605B
:1043F000231A526882189360A2688318A34202D0DD
:104400005E88002E00D070BD6E69A64200D16B613F
:10441000596061684018826070BDC046BC000020D1
:104420002872745F75696E74385F74202A296D650F
:104430006D203E3D20686561705F70747200000001
:10444000659100082872745F75696E74385F742016
:104450002A296D656D203C202872745F75696E7421
:10446000385F74202A29686561705F656E6400009A
:104470006D656D2D3E75736564203D3D20300000F7
:10448000F0B58DB00893174605910446149B580665
:1044900001D55BA000E055A007900122D80600D509
:1044A0009343D80701D0302000E0202003909807E4
:1044B0000025139904910028069302D402920095D6
:1044C00015E0002F07D458070CD418070025002842
:1044D000F4D5202007E001927F42002002902D2099
:1044E000009007E02B200090002002901546002F3E
:1044F0001ED001950025002F17D00A2638463146D8
:10450000FBF70AFF08990A2902D00F21394001E080
:104510004643B91B079A515C09AA515508990A29C3
:1045200000D038096D1C0746E5E70198089004E0C3
:10453000089509A83021017001251298049FBD42F9
:104540002946059E00DC3946401A1123069A1A4274
:1045500001D0039B12E0002801DC002300E00123CE
:10456000089A1A40801A039B012806DBB44201D244
:1045700020222270401E641CF6E7401E029A002A88
:1045800005D1B44201D2009A2270641C401E069AE2
:10459000D2060FD4012805DBB44200D22370401E9E
:1045A000641CF7E7401E05E0B44201D230222270BD
:1045B000491E641C8D42F7DB08E0B44204D209A90D
:1045C0004919491E097821706D1E641C002F08D0FE
:1045D000002DF2DC05E0B44201D220212170401E02
:1045E000641C0128F7DA20460DB0F0BD30313233BB
:1045F000343536373839616263646566000000001F
:104600003031323334353637383941424344454608
:10461000000000001CB514200A2100910190012027
:10462000830208A00949002201F086FC0446002804
:1046300004D107A00AA1C52200F01CF8204601F011
:10464000D9FE1CBD6D61696E000000000D400008C0
:1046500074696420213D2052545F4E554C4C00003B
:1046600072745F6170706C69636174696F6E5F69A9
:104670006E6974001CB513460A46014601A8002461
:10468000047008480468002C04D0084611461A46F5
:10469000A0471CBD04A000F00FFC01A80078002872
:1046A000FBD01CBD5810002028257329206173738E
:1046B000657274696F6E206661696C6564206174EF
:1046C0002066756E6374696F6E3A25732C206C6971
:1046D0006E65206E756D6265723A2564200A000071
:1046E000B0B504464C43204600F038FC054600288F
:1046F00004D000212846224600F03CFD2846B0BDEB
:10470000B0B5044C094DAC4202D201CC8047FAE767
:10471000B0BDC046E8950008B0B5044C044DAC42AD
:1047200002D201CC8047FAE7B0BDC046F49500083C
:1047300018960008014800687047C0469C06002093
:10474000B0B50446002805D195204200B34815496C
:10475000FFF790FF204600F0BDFF092806D0952006
:104760004000421CAF480F49FFF784FF2220215C24
:104770000020002906D022462232491E1170090667
:1047800002D0B0BDC043B0BD616B002500292846F2
:1047900005D020468847002801D0811DF1D125840D
:1047A000B0BDC0462A94000880B5092100F042FF40
:1047B00080BD00007CB50D460446002804D12E487B
:1047C0002E49E422FFF756FF204600F083FF092818
:1047D00004D02B482949E522FFF74CFFE08BC106A6
:1047E00010D4E16A002910D02046884700280BD059
:1047F000064600940190032022490122224B03F037
:10480000AFF836E0014603E0E08B10210143E1837D
:10481000208C090701D5010713D4010705D51B49D1
:104820002A460A400840904211D0226B002A0BD041
:104830002046294690470646002809D0B01D07D0DB
:1048400017E00620C64314E01048054025840026E2
:104850002220215C491C2154208C082202432284FE
:10486000C8B2884205D0FF22183209A00349FFF7D9
:1048700001FF30467CBDC0468E930008909400082E
:10488000E19300081C9400089D9300080F0F00009E
:104890006465762D3E7265665F636F756E74202168
:1048A0003D203000F8B517460E4604460B4D192042
:1048B0002877284624301421FBF7D1FC0848094901
:1048C000094AAA63E96328646F64AE640322284638
:1048D000214600F03DF80020F8BDC046A0060020AB
:1048E000F92600080D280008A5270008F8B51C4681
:1048F00015460E460746002805D12B20C200474822
:104900001249FFF7B7FE384600F0E4FE092806D04A
:104910002B20C000421C43480C49FFF7ABFE22206D
:10492000385C002808D02346BC6B002C08D03846E1
:1049300031462A46A047F8BD0520C043401D01E08E
:104940000520C04301F05CF90020F8BDD2930008B7
:10495000F8B50027FC43002812D00E460546009209
:104960000846FFF721FF00280AD1092128463246D0
:1049700000F0CCFE22202F540098E8832F843C4680
:104980002046F8BDB0B50C460546002805D1FF22EB
:10499000C43222480849FFF76DFE284600F09AFE0F
:1049A000092806D0FF20C430421C1E480249FFF7E8
:1049B00061FE6C620020B0BD3A940008F8B51C4658
:1049C00015460E460746002805D1FF2284321348BB
:1049D0001349FFF74FFE384600F07CFE092806D049
:1049E000FF208430421C0F480D49FFF743FE222070
:1049F000385C002808D02346FC6B002C08D03846D1
:104A000031462A46A047F8BD0520C043401D01E0BD
:104A10000520C04301F0F4F80020F8BD8E93000893
:104A20006E940008E193000880B5FBF763FB0F4923
:104A30004A88521C4A80FBF761FB80BD10B5FBF72A
:104A400059FB0A4C6188491E618009B2002902DDC8
:104A5000FBF754FB10BD00216180FBF74FFB606842
:104A60000028F7D000F0FCFE10BDC0460401002075
:104A7000F0B585B000287CD00446FBF73BFB06462A
:104A80008B20850000F0D0F9002809D03A483B4F30
:104A9000394600F011FA3A4839462A46FFF7EAFD4E
:104AA0003046FBF72BFBA00704D0AA1C35A03349E6
:104AB000FFF7E0FD3F4EF068A04202D83069A04207
:104AC00004D82A1D3C482D49FFF7D4FD7168002900
:104AD00001D020468847F068A0424AD83069A042F9
:104AE00047D901953046203000210391C9430490F5
:104AF00000F0F4FF27460C3FF520410125460A3D12
:104B00002888002802D0388888421DD002912BA026
:104B100000F0D2F93B882A882FA0394600F0CCF962
:104B20002888002805D1019A223237A01349FFF7BF
:104B3000A1FD38880299884206D0019A233235486F
:104B40000E49FFF797FD0299398003982880706914
:104B5000874200D27761F068083C21680818381A4B
:104B6000B1694018B0613846FFF716FC049800F0B0
:104B700071FF05B0F0BDC046518C00085D91000882
:104B80008E90000828282872745F75626173655FD3
:104B90007429726D656D292026202852545F414C7E
:104BA00049474E5F53495A45202D20312929203D40
:104BB0003D203000BC000020BE900008746F2066CD
:104BC00072656520612062616420646174612062A5
:104BD0006C6F636B3A0A00006D656D3A2030782582
:104BE0003038782C207573656420666C61673A20D4
:104BF00025642C206D6167696320636F64653A20CA
:104C00003078253034780A006D656D2D3E757365FA
:104C1000640000009090000880B502F0D9FB02F01B
:104C200007F97D20C1000C480068FBF775FB401EAA
:104C3000010E08D1094948600948FF220270072087
:104C4000086000208860FCF795FEFFF759FD0548D5
:104C5000054901F077F880BD0C00002010E000E06D
:104C600023ED00E0D02400200040002080B5FCF7B8
:104C700073FEC0B280BD000080B50246002002A1D4
:104C8000FCF718FF80BDC046257300000446C169CB
:104C90000FA0134DA847A16912A0A847616915A0EC
:104CA000A847216917A0A847E1681AA0A847A168EA
:104CB0001CA0A84761681FA0A847216821A0A84799
:104CC0002448016824A0A847FEF7F4FEFEE7C0468A
:104CD0007073723A203078253038780A000000006E
:104CE000B94E00082070633A203078253038780AB1
:104CF00000000000206C723A203078253038780AA5
:104D0000000000007231323A203078253038780ABD
:104D1000000000007230333A203078253038780AAD
:104D2000000000007230323A203078253038780A9E
:104D3000000000007230313A203078253038780A8F
:104D4000000000007230303A203078253038780A80
:104D5000000000000801002068617264206661752F
:104D60006C74206F6E207468726561643A202573DC
:104D70000A00000080B5074801682F220A4302603C
:104D800000BF00BF00BF04A004490022FFF78AFD56
:104D900080BDC0462C10024070696E00D47C0008B3
:104DA000F0B5141D072294432246403A3F25ED43B7
:104DB0000D4E002D02D066512D1DFAE725461C3DF3
:104DC00000262746203F39602E606E60AE60EE60A0
:104DD000211F01252D060D602146083908600C3C75
:104DE00023601046F0BDC046EFBEADDE10B5E12039
:104DF000400200242146FDF7BBF84B2080012146EC
:104E0000FCF7C2FC204610BD10B5FBF773F9044651
:104E100012480178491C01704068002800D0804782
:104E20002046FBF76BF910BD10B5FBF763F90B4992
:104E30000C78FBF763F9204610BDC04610B5FBF7B0
:104E400059F9044605480178491E01708068002818
:104E500000D080472046FBF751F910BDB00000207C
:104E600080B500681C3801F049FA80BD70B516465F
:104E70000C460546084601F011FB002E14D0012E09
:104E800019D121463D3128460068A8420CD0212284
:104E9000825C0B789342F7D2416822461C320A604A
:104EA000E0612162426070BD686821461C3101608A
:104EB000E5612062696070BD83B078B5054605A8DC
:104EC0000EC005AB00931048FF2421462A4601F08E
:104ED000B3FD03461B4D286800280DD0068C4021E9
:104EE00031430184FF2B00D323460021064AFFF7FC
:104EF00065FD2868068402E00348FFF7BDFE78BC24
:104F000001BC03B00047C04664100020F8B500287B
:104F100013D004460B4E3568002D0FD02F8C402047
:104F200038432884204600F0DEFE03460021284650
:104F30002246FFF743FD30680784F8BD2046FFF79F
:104F40009BFEF8BD9C0600200021C9430246491C77
:104F500012688242FBD1084670470000F0B587B066
:104F60000027002853D00446FBF7C4F80546FFF796
:104F70005BFF00280AD05748574E3146FFF79CFF89
:104F80002320C20055483146FFF774FB2846FBF743
:104F9000B5F8E41C03208443514DA868844236D8F8
:104FA0002846203000210491C943059000F096FD69
:104FB0000C2C00D80C24A968E868069402910B1BFD
:104FC000696903910F1A06999F421CD23D46C61982
:104FD00077687288002AF7D12A460C32BC1A8C42B4
:104FE000F2D306990B460C330193F5235B0104932E
:104FF00018318C420ED2019C012272807A1B384DEE
:10500000AB699A181EE0059800F024FD049F38460D
:1050100007B0F0BD069952180499815283185F6059
:1050200000245C8072609D60012474805B68029C37
:105030000C34A34201D0C3189A60294DAA69019982
:105040000C468A18AA61EB699342039900D2EA617F
:10505000049A32802322D7008E4213D12A694B88CA
:10506000002B05D0914203D0496841186961F6E7E9
:10507000914207D0002B05D03A466A3219A0164952
:10508000FFF7F8FA059800F0E5FCA01929698842B5
:105090003C4605D922466E321C480F49FFF7EAFA12
:1050A00037460C37B80705D022466F3218480A49F0
:1050B000FFF7E0FAB00705D0703416A00649224683
:1050C000FFF7D8FA2A68002AA1D0384606999047F7
:1050D0009DE7C046518C0008B49000088E900008EF
:1050E000BC00002028286C66726565203D3D206864
:1050F0006561705F656E6429207C7C2028216C6668
:105100007265652D3E757365642929001A91000842
:105110004790000828282872745F75626173655F84
:1051200074296D656D292026202852545F414C4911
:10513000474E5F53495A45202D20312929203D3DB6
:105140002030000010B581420AD28B18834207D963
:10515000491E431E002A0CD08C5C9C54521EF9E759
:105160000346002A05D00C781C705B1C491C521E9B
:10517000F7E710BD10B5042A14D30323034011D15F
:10518000CBB20C4C5C4303460F2A08D91C605C6010
:105190009C60DC60103A1033F6E710C3121F042A3B
:1051A000FBD204E0034602E019705B1C521E002A89
:1051B000FAD110BD01010101F8B514460E460546AD
:1051C00007462637002804D10A480BA10E4AFFF7EC
:1051D00051FA03212846324600F098FA0020A862CE
:1051E0000121A98429461C31E9612962FF21398006
:1051F0006C74F8BD078D000872745F6D7574657806
:105200005F696E69740000001D020000F8B5044675
:10521000CB208500002C04D19E4846492A46FFF742
:1052200029FA204600F056FA032804D06A1C9A484E
:105230004049FFF71FFAFAF75DFF064601F0A0F8B4
:10524000002809D191483B4F3946FFF735FEAA1D8A
:10525000BC483946FFF70EFAFAF74CFF0746FFF74E
:10526000E3FD002808D0B5483249FFF725FEAA1D06
:10527000B4483049FFF7FEF93846FAF73FFF3046A9
:10528000FAF73CFF01F07CF80746FAF733FF0546D2
:1052900029480168002901D020468847A06A874232
:1052A00007D00220C043841CBC632846FAF726FFBF
:1052B0000AE0264626367078401E7070000605D03B
:1052C0002846FAF71BFF00242046F8BD3D20385C35
:1052D0003178814204D002213846324600F0DAFDAE
:1052E000E16920461C30814212D00A461C3AA26273
:1052F0002122895C31707178FF290DD0491C7170B1
:10530000FFF7AEFD2846FAF7F9FE00F0A9FADAE752
:10531000A08C0A49884205D12846FAF7EFFE022000
:10532000C443D1E70021A162FF213170401CA08459
:10533000C6E7C046A58D00086C110020FFFF0000E5
:10534000FEB5044601910291FAF7D4FE07465320B8
:10535000C60001F015F8002809D14C484C4D2946EB
:10536000FFF7AAFDD04829463246FFF783F9FAF73E
:10537000C1FE0546FFF758FD002808D0C84844493B
:10538000FFF79AFDC84842493246FFF773F92846AD
:10539000FAF7B4FE3846FAF7B1FE002C04D1F21C3D
:1053A0003C483B49FFF766F9204600F093F9032893
:1053B00004D0321D38483649FFF75CF900F0E0FFB1
:1053C0000746FAF797FE054634480168002901D0E0
:1053D00020468847214626310026BE63A06AB8428F
:1053E00008D0A28C002A1CD0A762501EA0843D20A9
:1053F000385C08704878FF2805D12846FAF77EFE09
:105400000220C5430BE0401C48702846FAF776FEA0
:1054100023480168002901D02046884735462846A0
:10542000FEBD0199002929D000953D21425C795C9F
:10543000914204D23A463D32022100F02BFD627CBB
:1054400020461C303946FFF711FD0198012809DB81
:105450003D465435002102AA284601F05BF9284652
:1054600001F02AFA0098FAF749FE00F0F9F9BD6B4D
:10547000002DD4D1FAF73EFE0546C6E70220C1430F
:1054800028464D1CBD63FAF739FEC8E7788C000842
:10549000438D0008078D0008C28F0008741100209A
:1054A00070110020F8B500910546FAF723FE064674
:1054B000DF204700FFF7B8FC002809D07848204CCF
:1054C0002146FFF7F9FC784821463A46FFF7D2F823
:1054D0003046FAF713FE284600F0E8F806460028A2
:1054E00004D13A1DA9481649FFF7C4F8F068FFF740
:1054F00035FD074600281ED0F268002438462146B4
:10550000FFF738FE7C743D7410223846009900F095
:1055100004FCA4480168002901D038468847FAF7FE
:10552000E9FD716879613A4614324A607260311D52
:10553000B961FAF7E3FD3846F8BDC046518C000862
:10554000BC9100088E90000810B50446002805D1D3
:10555000F920420013481449FFF78CF81020205618
:10556000002806D5F9204000421C10A00E49FFF784
:1055700081F82F480168002901D020468847002083
:105580002074FAF7B7FD6169A2694A60A2691160E7
:10559000214614316161A161FAF7B0FD2046FFF7A1
:1055A00067FA10BD9B910008CF91000821286F6217
:1055B0006A6563742D3E7479706520262052545FAD
:1055C0004F626A6563745F436C6173735F537461A8
:1055D000746963290000000010B50446002805D155
:1055E000CF2042000C480DA1FFF744F81048016895
:1055F000002901D02046884700202074FAF77AFD60
:105600006169A2694A60A269116021461431616131
:10561000A161FAF773FD10BD9B91000872745F6F72
:10562000626A6563745F64657461636800000000AA
:1056300068110020F8B50446084600F037F8002647
:10564000002C2BD00546002828D0FAF753FD06463B
:10565000FFF7EAFB00280AD0E948124F3946FFF766
:105660002BFC91208200E8483946FFF703F83046CA
:10567000FAF744FDFFF7D8F92D1D2F463F68AF42DA
:1056800009D03E46143E10223046214600F032FB3F
:105690000028F3D100E00026FFF7D0F93046F8BD2E
:1056A000518C0008AD9100088E90000810B58F2134
:1056B000CB4307491A46103208D0CB1890241B5D03
:1056C00083421346F7D18818803010BD002010BDEA
:1056D0001000002010B50446002804D1044805A19C
:1056E000094AFEF7C7FF217C7F20084010BDC04655
:1056F0009B91000872745F6F626A6563745F67658F
:10570000745F74797065000027020000FEB5029294
:10571000044601910846FFF7C9FF05469B20470054
:10572000002D04D119481A493A46FEF7A3FFFFF7A6
:105730007BF92E1D35462D68B5420AD0284614380F
:10574000A042F8D13A460E3212A01149FEF792FF5C
:10575000F1E78020019D0543FFF770F925741022C1
:105760002046029900F0D9FA0E480168002901D0BC
:1057700020468847FAF7BEFC316861612246143240
:105780004A603260A661FAF7B9FCFEBD8491000858
:10579000E09100086F626A20213D206F626A6563B4
:1057A000740000006411002010B50446002805D1E3
:1057B00085208200034804A1FEF75CFF207CC0091D
:1057C00010BDC0469B91000872745F6F626A65638A
:1057D000745F69735F73797374656D6F626A656313
:1057E0007400000070B50C460546084EB06C0028E9
:1057F00005D1074807A19D22FEF73CFFB06C036866
:10580000024829462246984770BDC046A00600209F
:10581000D594000872745F70696E5F6D6F64650087
:1058200070B50D460446084EB06C002805D10748F7
:1058300007A1A322FEF71EFFB06C4368EAB202483C
:105840002146984770BDC046A0060020D5940008A8
:1058500072745F70696E5F77726974650000000032
:10586000F8B5FAF747FC04464D4F7888002803D076
:105870002046FAF743FCF8BDF868FCF7D3FE401E5B
:10588000C100464A555829461C397E68B142EFD0BE
:1058900079603870BA68002A01D0304690470835E0
:1058A000243607480078002804D030462946FAF705
:1058B00028FCDDE730462946FAF723FCD8E7C04646
:1058C000B0000020F8B5044605463C35002805D157
:1058D000FF2218320E480FA1FEF7CCFEFAF70AFCA1
:1058E0006978C9002D4A51184A68226223461C3340
:1058F0001360226C2A4EF7681743F7602A78F02667
:105900001640721C2A704B60E161FAF7F7FBF8BD94
:10591000EF91000872745F7363686564756C655F0E
:10592000696E736572745F7468726561640000000B
:1059300010B50446002805D1FF2246320F4810A1B9
:10594000FEF798FEFAF7D6FBE169226A4A60226AFE
:10595000116021461C31E16121623D21615CC90079
:105960000E4A53185158994204D1216C0C4AD368FD
:105970008B43D360FAF7C2FB10BDC046EF9100081D
:1059800072745F7363686564756C655F72656D6F73
:1059900076655F7468726561640000007C110020A8
:1059A00004010020F8B516460D460090FAF7A2FB58
:1059B0000446FF270E37FFF737FA002808D08E4835
:1059C0001049FFF779FA8B480E493A46FEF752FE26
:1059D0002046FAF793FB280C04D07A1C1C4809498E
:1059E000FEF748FE02200099FFF75CFD002805D075
:1059F0008584467401461C31C1610162F8BDC04610
:105A0000518C0008C38D00088E900008F8B51C4624
:105A100016460F460546002804D171480B49D2228C
:105A2000FEF728FE300C04D009480849D322FEF7BF
:105A300021FE022128463A46FFF768FEAE8428463A
:105A40001C30E86128626C740020F8BD428F0008A9
:105A5000188D0008F8B50446002805D1FF22B83299
:105A60005F481B49FEF706FE2046FFF733FE02287B
:105A700006D0FF20B830421C5B481549FEF7FAFDFE
:105A800014480168002901D02046884725461C3566
:105A9000FAF730FB0646E769AF4203D02846FFF726
:105AA000DFF90BE0A08C0C49884205D13046FAF7AB
:105AB00025FB0220C44309E0401CA0843046FAF7CD
:105AC0001DFB0024AF4201D0FFF7CAFE2046F8BDFF
:105AD000968D00086C110020FFFF0000FEB50D46FA
:105AE0000446029153208700002C04D13C483D49D4
:105AF0003A46FEF7BFFD2046FFF7ECFD022804D032
:105B00007A1C39483749FEF7B5FD38480168002945
:105B100001D020468847FAF7EDFA0646A08C002807
:105B20000CD0401EA0843046FAF7E8FA33480168EA
:105B30000025002951D0204688474EE0002D47D04F
:105B4000FAF7D8FA019000F01BFC002809D1284888
:105B50002449FFF7B1F93A4621329F482149FEF71F
:105B600089FDFAF7C7FA0090FFF75EF9002809D01F
:105B700097481C49FFF7A0F92137974819493A4639
:105B8000FEF778FD0098FAF7B9FA0198FAF7B6FA35
:105B900000F0F6FB07460020B863627C20461C300C
:105BA0003946FFF763F9012D09DB3D4654350021E5
:105BB00002AA284600F0AEFD284600F07DFE3046E1
:105BC000FAF79CFAFFF74CFEBD6B002D05D1ADE74F
:105BD0003046FAF793FA0120C5432846FEBDC04679
:105BE000C78C0008378D0008518D00087411002003
:105BF000788C00088E900008518C000870110020ED
:105C000010B50446FFF710F9002802D004480460DC
:105C100010BD00F0B5FB0028F8D0846310BDC0466D
:105C2000880200201CB507A0094CA04709A0A04786
:105C300011A0009013A0032101220523A04719A061
:105C4000A0471CBD0A205C207C202F0A0000000019
:105C5000B94E00082D205254202D20202020205401
:105C60006872656164204F7065726174696E672047
:105C700053797374656D0A005365702020352032A6
:105C800030323400202F207C205C20202020202552
:105C9000642E25642E2564206275696C642025734A
:105CA0000A0000002032303036202D2032303230D1
:105CB00020436F707972696768742062792072740A
:105CC0002D746872656164207465616D0A0000005E
:105CD00081B0C0B5039303AB009300F0ADFE88BC68
:105CE00002BC01B008470021425C491C002AFBD1DC
:105CF000481E704770B50023002A0BD00C78057839
:105D00002C1B260607D1002D1C4604D0491C521E10
:105D1000401CF0E71C4660B270BD10B5002A09D0E7
:105D200003460C781C70002C05D05B1C521E491CCD
:105D3000002AF6D110BD01218A42FBD000245C5418
:105D4000491CF9E7F8B50F4600900320C5430C46FF
:105D50002C40FAF7CFF90646FFF766F8002808D07E
:105D60001B481C49FFF7A8F81B48D2221949FEF727
:105D700081FC3046FAF7C2F9192C009905D3C81CEA
:105D800028402246183A824204D218A03A46FFF729
:105D900093F8F8BD211A0A46183A104DAA60F52268
:105DA00052010C3900230260416083600C3C616049
:105DB000E8602C610A482060A8680C30A060284682
:105DC000203008A10122FFF721FEE8686861F8BDD4
:105DD000518C0008709100088E900008BC000020D3
:105DE000A01E010068656170000000006D656D20F7
:105DF000696E69742C206572726F722062656769C2
:105E00006E206164647265737320307825782C206D
:105E1000616E6420656E64206164647265737320D2
:105E2000307825780A0000001348002141802022A4
:105E3000124B002A04D01B605B600833521EF8E747
:105E400041601F22027002461032C160026142614D
:105E50007047C04610B5084CE068FCF7E3FBC00093
:105E6000064940180838006801461C39616008304E
:105E7000FAF77FF910BDC046040100207C11002014
:105E8000024801460C31C160016170471C010020CD
:105E900070470000F8B515460E460446002804D1A8
:105EA00091482349234AFEF7E5FB2046FFF712FC01
:105EB000012805D01F48421C8D481D49FEF7DAFB1A
:105EC000002E19D0012E1BD0022E2ED127463C3792
:105ED000FAF710F9064638780F210140012918D148
:105EE0002046FFF725FD2878787001218140216444
:105EF0002046FFF7E7FC11E0204600F07BFA14E0B3
:105F00002046FFF751FC01280CD1204600F0A0F8F4
:105F10000BE0287878700121814021643046FAF73F
:105F2000EDF802E0204600F02DF80020F8BDC04654
:105F30009E92000877020000F0B585B01F460492DB
:105F40000D4601460120FFF7ADFA0024002815D0C8
:105F500006463846FFF702F800280CD003460B9897
:105F60000A9900970191029030462946049AFCF75D
:105F700083FC344602E03046FFF7E6FA204605B0DF
:105F8000F0BD000070B50446CF204500002C04D1C0
:105F90001D481E492A46FEF76DFB2046FFF79AFB77
:105FA000012804D06A1C1A481849FEF763FB2046F2
:105FB000FFF7FAFB002804D0AA1C16A01349FEF72D
:105FC00059FB3C20215C0F20084004D0042819D044
:105FD0002046FFF7ADFC25463C352046FCF7A8FCE3
:105FE0002046543000F0ECFB26461C36FAF782F8C7
:105FF0008E490A68566004232B700E60E2612162AC
:10600000FAF77CF8002070BDEF9100086692000856
:106010000192000872745F6F626A6563745F6973EE
:106020005F73797374656D6F626A65637428287233
:10603000745F6F626A6563745F7429746872656106
:106040006429203D3D2052545F46414C5345000099
:10605000B0B50446FF253A35002804D1224823492B
:106060002A46FEF707FB2046FFF734FB012804D041
:106070006A1C1F481D49FEF7FDFA2046FFF794FBF6
:10608000002804D1AA1C1BA01849FEF7F3FA3C20F3
:10609000215C0F20084004D0042822D02046FFF7BE
:1060A00047FC25463C352046FCF742FC2046543050
:1060B00000F086FB042028702046FFF775FB0128BE
:1060C00003D12046FFF788FA0BE025461C35FAF786
:1060D00011F856490A6855600D60E2612162FAF7CD
:1060E0000DF80020B0BDC046EF910008779200087F
:1060F0000192000872745F6F626A6563745F69730E
:106100005F73797374656D6F626A65637428287252
:10611000745F6F626A6563745F7429746872656125
:1061200064290000B0B5DC480568F9F7E3FF0446D0
:106130002846FCF7FDFB2846FFF7FAFB3C2004212C
:1061400029542846543000F03BFB2846FFF72CFB2F
:10615000012803D12846FFF73FFA07E033480168DA
:106160002A461C324A600260E9612862FFF778FB28
:106170002046F9F7C3FFB0BD0024074D2646042E84
:1061800006D0B0002858002800D08047761CF6E7DB
:1061900000F004F8F2E7C046C40F002070B5F9F72C
:1061A000A9FF0446FEF740FE002809D013A01D4DAC
:1061B0002946FEF781FE1CA093222946FEF75AFAD3
:1061C0001A4E2046F9F79AFFF9F794FF044635680E
:1061D000B5420ED003CD4160083D696808602D606E
:1061E0006D606869FEF744FC1C3D2846FFF7ACF97A
:1061F000E7E72046F9F782FF70BDC04646756E633B
:1062000074696F6E5B25735D207368616C6C206EC2
:106210006F74206265207573656420696E20495330
:10622000520A00003B8C00083000000014010020DE
:106230001FB5202003901F200290084800900120E5
:1062400000020190064C07A1084A0023204600F0F6
:106250000FF8204600F0CEF81FBDC0468012002087
:10626000340F00207469646C6500000079610008D7
:10627000F0B587B0069305920A4607460C9E0028A3
:1062800006D1124812491446E922FEF7F3F92246D4
:106290000F9804900E9C0D9D002E06D10DA00C4968
:1062A0000392EA22FEF7E6F9039A01213846FFF746
:1062B0002DFA009501940498029038460599069AA3
:1062C0003346FCF7D9FA002007B0F0BDEF91000883
:1062D000D2920008737461636B5F7374617274208F
:1062E000213D2052545F4E554C4C000080B500F0CB
:1062F0009BF900F049F8002080BD000070B504460D
:10630000002804D19F481B491B4AFEF7B3F92046D9
:10631000FFF7E0F9012805D01748421CAA481549A3
:10632000FEF7A8F93C20205C0F210140002502293E
:106330001CD1F9F7DFFE0646E069216A4160216A57
:10634000086020461C30E06120622046543000F096
:1063500035FB3046F9F7D2FE2046FFF7B3FA07487F
:106360000168002903D02046884700E0ED43284615
:1063700070BDC04655920008F70200007C12002054
:10638000A74800687047C046F8B50090F9F7B2FE1C
:106390000546A3480468002C05D1FF22FC32794849
:1063A0001349FEF767F92046FFF794F9012806D054
:1063B000FF20FC30421C84480D49FEF75BF9204663
:1063C00000F06CF82746543700266A4638463146B6
:1063D00000F0A0F9384600F06FFA2846F9F78EFE73
:1063E000FFF73EFAA06B801C00D1A6630020F8BD29
:1063F000B092000870B50446FF250E3506463C36BF
:10640000002804D1144815492A46FEF733F930789C
:10641000000704D06A1C12A01049FEF72BF9204691
:10642000FFF758F9012804D0AA1C67480B49FEF76A
:1064300021F902203070B078707001218140216410
:106440002046FFF75BFF76480068002801D0FFF781
:1064500007FA002070BDC046EF910008C092000806
:10646000287468726561642D3E73746174202620FF
:1064700052545F5448524541445F535441545F4D18
:1064800041534B29203D3D2052545F5448524541D1
:10649000445F494E4954000008010020F8B5044605
:1064A000002804D137481A491A4AFEF7E3F8204673
:1064B000FFF710F9012805D01648421C424814493C
:1064C000FEF7D8F83C20205C0F210140002501296F
:1064D0001AD127463C37F9F70DFE06462046FFF74E
:1064E00027FA3878F0210140881C38702046543053
:1064F00000F064FA3046F9F701FE07480168002908
:1065000003D02046884700E0ED432846F8BDC0464A
:1065100043920008CD02000080130020B0B504466D
:10652000174D002804D1174817492A46FEF7A2F84C
:106530003C20205C0F210140022904D06A1C13A0DA
:106540001149FEF797F82046FFF7C4F8012804D058
:10655000AA1C1D480C49FEF78DF8E069216A4160CC
:10656000216A08600120C043A06320461C30E0611E
:1065700020622046FFF7A6F9FFF772F9B0BDC046CA
:1065800023030000EF910008E1920008287468726C
:106590006561642D3E7374617420262052545F54EB
:1065A00048524541445F535441545F4D41534B2938
:1065B000203D3D2052545F5448524541445F53555D
:1065C0005350454E4400000001920008B0B5F9F761
:1065D00091FD134909683C228A5C0F231340012B6B
:1065E00019D1CA690B6A9A4215D00C463C340D4643
:1065F0001C3553600B6A0D621A606278D200094B39
:106600009A1853681D60CA610B625560F9F776FDF0
:10661000FFF726F901E0F9F771FD0020B0BDC04693
:10662000080100207C110020C117084370470000BA
:106630000A4800687047C04680B508480168491C90
:106640000160FFF79DFE016D491E016503D1C16C1C
:106650000165FFF7BBFF00F003F880BD8813002041
:10666000FEB501A801900290FFF7E2FF0646F9F798
:1066700041FD0090D048C5680C30854243D0686920
:10668000301A234988423ED82C461C3CCA4801682F
:10669000002901D02046884703CD4160083D696844
:1066A00008602D602F460B3F3878810702D4FE2109
:1066B0000840387001984560286001A8686001951D
:1066C000A968E8688847FFF7B3FF0646BA484168FB
:1066D000002901D02046884701A801998142C9D0EC
:1066E00003CD4160083D696808602D606D603878B1
:1066F0008107BFD5C107BDD0FE21084038702046B4
:1067000000F0DAF8B6E70098F9F7F8FCFEBDC046ED
:10671000FEFFFF7F70B515460E460446002805D1E2
:10672000FF22DA32C0481949FDF7A4FF2046FEF7E0
:10673000D1FF0A2806D0FF20DA30421CBC4813499A
:10674000FDF798FFF9F7D6FC042E1BD87E44367966
:106750007600B744020A0C1005002968E16211E0D6
:10676000617CC9070CD100210BE0E16A09E0617C82
:10677000FD220A4002E0617C02220A43627401E0C9
:1067800001212960F9F7BAFC002070BD24930008AC
:1067900070B51C4615460E4601460A20FEF782FEDD
:1067A00000280CD004990022FE230B4043740146BC
:1067B0001C31C161016246628562C462026370BDC0
:1067C00010B50446002804D117481849DD22FDF70A
:1067D00051FF2046FEF77EFF0A2804D014481349D3
:1067E000DE22FDF747FF2046FEF7DEFF002804D13A
:1067F00010A00E49DF22FDF73DFFF9F77BFCE169B0
:10680000226A4A60226A1160617CFE220A40627438
:1068100021461C31E1612162F9F770FC2046FEF748
:10682000DBFE002010BDC046F39200081493000860
:106830004393000872745F6F626A6563745F697383
:106840005F73797374656D6F626A6563742826740B
:10685000696D65722D3E706172656E74290000006D
:10686000FEB5029301920F460546099E089C00283A
:1068700004D10C480CA1C922FDF7FCFE0A212846D0
:106880003A46FEF743FF0020FE210E406E74294673
:106890001C31E9612962019969620299A962EC627D
:1068A0002863FEBDF392000872745F74696D6572AF
:1068B0005F696E6974000000FEB50446FF2642362B
:1068C000002804D12E482F493246FDF7D3FE20463A
:1068D000FEF700FF0A2804D0721C2B482949FDF757
:1068E000C9FEF9F707FC0290E069216A4160216A5C
:1068F0000860607CFE210140617420461C30E0612C
:106900000190206221480168002901D02046884773
:10691000E06A1F4DA84205D310361EA01949324621
:10692000FDF7A8FEFFF784FEE16A0A1822632248F9
:1069300001460C3103690126F0070DD008460026F8
:10694000984207D0014600684769BF1AF7D0AF42A6
:10695000F5D2F1E71946EFE70868E061019A426075
:10696000154B9868401C98600A602162607C012188
:10697000014361740298F9F7C1FB0020FEBDC046D7
:10698000F39200087F9300084393000870110020E1
:10699000FFFFFF7F74696D65722D3E696E69745FDC
:1069A0007469636B203C2052545F5449434B5F4DE4
:1069B0004158202F203200001C010020B0B50446B1
:1069C000002805D1DB20420017481849FDF752FE88
:1069D0002046FEF77FFE0A2806D0DB204000421C3E
:1069E00013481249FDF746FE0025607CC00701D11F
:1069F000ED4316E00F480168002901D02046884782
:106A0000F9F778FBE169226A4A60226A1160617CC9
:106A1000FE220A40627421461C31E1612162F9F7CD
:106A20006DFB2846B0BDC046F392000835930008C0
:106A3000439300086C110020F0B58DB00B93044611
:106A40000C9200230893DF4305910029069701D497
:106A500005996718E1430391049407971078252856
:106A600007D0002800D133E1BC4200D22070641C62
:106A70002AE1501C089F0178202909D0232909D038
:106A8000302909D02D2909D02B290BD1042106E06A
:106A9000082104E0202102E0012100E010210F4341
:106AA000401CE8E70C900A46303A092A05D80CA8A1
:106AB00000F0ACF906460C980DE02A290AD1401CDA
:106AC0000C900B9940C9002E0B9104D510210F4357
:106AD000764200E0069E03782E2B0CD1411C0C91CF
:106AE00042781346303B092B09D80CA800F08EF9E8
:106AF00002460C990CE0014606980A900CE02A2AFE
:106B000005D1811C0C910B9804C80B9000E0069AEB
:106B1000D01782430A920B78042018436C2805D1C1
:106B2000481C0C904A780146184601E000201A469D
:106B300015466F3D0A23092D17D9252A5BD0582AFF
:106B40005FD0692A1FD0642A1DD0632A20D1F8069D
:106B500000D5A2E0079F022E00DAA0E0BC4201D2DD
:106B600020202070761E641CF5E709930346C0467A
:106B70007D442D796D00AF44041B0B0B300B490B8A
:106B80000B47082041E009930346022007433DE0FC
:106B9000079FBC4203D2252020700C990A78601C04
:106BA000002A00D18DE0B84200D20270A41C8BE014
:106BB0000B9804C80B900A980190701C00D108260D
:106BC0000096414241410F43F8B202901023204603
:106BD000079F3946FDF754FC75E00B9A02CA00295D
:106BE00000D144A100230B929E422BD0C85C002808
:106BF00029D05B1CF8E7079FBC4200D337E725206C
:106C000034E703464020074310200990682B04D046
:106C10006C2B0B9D2A68099B06E00B980288B8072D
:106C2000099B00D512B20B9DF8B200960A9901910A
:106C300002902046079F3946FDF722FC04462D1D91
:106C40000B9541E033460A988342024600DC1A461F
:106C5000002800DC1A46F80609D4079FB24208DA79
:106C6000BC4201D220202070761E641CF6E7079FEC
:106C700000E0761E0023E01893420BDAB84201D2FE
:106C8000CD5C05705B1CF6E7B84201D22021017093
:106C9000761E401CB242F7DB15E0079F00E0761E2F
:106CA0000B99BC4201D208682070091D641C022E99
:106CB00005DBBC4201D220202070761EF6E70B9146
:106CC00002E0491E0C9104460C98421C0C92C5E649
:106CD00005980028039900D40146002905D0BC423C
:106CE000204600D3781E089901700498201A0DB030
:106CF000F0BDC046284E554C4C29000010B501216E
:106D00008A02184803460C3B1C6814431C6000BFF1
:106D100000BF00BF0A071C6814431C6000BF00BF0F
:106D200000BF0A02104B1C6814431C600368022455
:106D30001C430460036810241C4308239C43046024
:106D400003680B43036003685B07FCD503231B0246
:106D500004689C4314430460C90302680A43026048
:106D600010BDC04640100240007000400020704737
:106D700000207047002070470020704780B5F9F769
:106D8000B9F9FDF749FFFEF74DFFFFF779F8FFF777
:106D90004BF8FDF73FFCFFF77BF8FFF749FAFFF7E9
:106DA00059F8002080BD000010B5044606A0FEF78B
:106DB00083F8FBF78DFEDF204000221804480549C8
:106DC000FEF77AF810BDC0461B5B324B0D00000089
:106DD000368C00089C070020F8B5044609A50AA6D1
:106DE00007463F68A7420BD039461C392846FEF7B4
:106DF00063F83868A042F4D03046FEF75DF8F0E75B
:106E0000F8BDC046257300002F00000010B50268D1
:106E100000211378303B092B08D8531C03600A2447
:106E20004C431178611830391A46F2E7084610BD14
:106E30000448016804220A430260016801220A43EF
:106E40000260704710E000E0B0B5026814215143C1
:106E5000154A8C580A4B23404468C5682543046989
:106E60002C434569254384692C431C438C508B5823
:106E70001F242404A3438068000418438850B0BD35
:106E80000FE7FFFF10B5016814224A430649531863
:106E9000C4685C6044689C608068D8605058012376
:106EA0000343535010BDC04608000240F8B50D46DC
:106EB00006460524204600F021F8002800D0F8BD41
:106EC000284F386806210091884330433860022EED
:106ED00007D17F20000239688143280208433860C7
:106EE00000E032243868082101433960204600F070
:106EF00005F83968009A91433960F8BD10B5044629
:106F0000F34800687D21C900F9F706FA6043411C87
:106F100007480268D20303D5491EFAD1042010BDE8
:106F20000168044A02601C200840411E884110BDCF
:106F3000102002401C000001F8B50D460646012451
:106F40002046FFF7DBFF002800D0F8BD054F38686A
:106F50002043386035602046FFF7D0FF3968A143F1
:106F60003960F8BD14200240FEB50D4601900024A2
:106F7000019E29680846E0402CD00120A040014035
:106F800026D0084648436A680346534303274743CD
:106F900002942C463568BD431D433560A3684343C6
:106FA000F568BD431D43F5602546029C022A0FD1BA
:106FB0002A69FF2909D8404342430F214143019BDD
:106FC000186A88431043186202E0019800F00EF836
:106FD000641CCEE76868401E012806D8E86848436C
:106FE000019B5A688A4302435A60FEBD090A49431D
:106FF00049434A430F234B43416A9943114341623A
:10700000704770B50E46044600680125A84320600D
:10701000280321688143F06808432060032041026F
:1070200022688A43716911432160010362688A43BF
:10703000316911436160E16A0F22914332680A436A
:10704000E2620002A1688143B0690843A060B168B0
:10705000204600F01BF8002815D120680C21884339
:107060007168014321602068216801220A4322607F
:10707000010702D5E1698902FCD50025400702D548
:10708000E0694002FCD5284670BD000070B50D4691
:1070900004460026214884420ED0214884423046CE
:1070A0001ED1204800680005810F1F4879440979E6
:1070B00049008F440D1015131A4800688005810F90
:1070C0001948C0467944097949008F4401040907E9
:1070D00000F048F804E000F081F801E00120C0036E
:1070E000E16A0907C90E11A2515AF9F715F9010E03
:1070F00000026A08801871412A463346F9F766F89B
:1071000010494118104A914206D8E1680F4A0A40D6
:107110000243E260002070BD012070BD0084004089
:10712000008000403C1002400024F40001000200F6
:107130000400060008000A000C00100020004000B7
:107140008000000100FDFFFFFFFC0F000000F0FFCA
:1071500080B500F043F8BC4909684905490FC840AB
:1071600080BDC04610B507200403FFF7F1FFB64904
:1071700009682140090B032901D3C91E00E0002141
:10718000C84010BD10B507200404FFF7E1FFAE4969
:1071900009682140090C032901D3C91E00E0002120
:1071A000C84010BD10B50C4C2068C00701D01C4869
:1071B00000E01C4821680906C90E00D1202148437F
:1071C00021684905490F00D10821F9F7A5F8216880
:1071D0004903890FC84010BD0C10024080B50F480C
:1071E00081688906490F491E03290AD80C48C04600
:1071F0007944097949008F4409010A0DFFF7D2FF4C
:1072000080BD0068C004810F0648C84080BD7D2055
:10721000000280BD0120C00380BDC04600100240B6
:1072200000127A000024F400B0B50446384DCA209C
:1072300028605320286000F017F8002801D00420AF
:107240000EE0A0782178490308186178090201430B
:10725000E0780004084329462039086000F020F84F
:1072600000212960B0BDC04670B519480568194EA7
:1072700030680024400610D430688021014331601A
:107280007D20C1002846F9F747F8681AC0433168E5
:10729000490602D4401CFAD30424204670BDC046DF
:1072A000B0B50B4804680B4D2868802188432860DE
:1072B0007D20C1002046F9F72FF8601AC0432968E5
:1072C000490603D5401CFAD30420B0BD0020B0BD50
:1072D0000C0000200C280040B0B504460C4DCA201C
:1072E000286053202860FFF7BFFF002801D004204A
:1072F0000BE020780004617809020818A178401892
:10730000294624390860FFF7CBFF00212960B0BD72
:1073100024280040B0B50D460446124884420BD0E4
:107320001148844205D01148844202D0104884425A
:1073300015D1FFF717FF01E0FFF724FF21680904CB
:10734000C90F8840690840182946F8F7E5FF01464B
:107350001039084A914202D8E0600020B0BD0120F7
:10736000B0BDC0460038014000440040004C004021
:1073700000480040EFFF0000B0B501231A03046885
:107380009443CA6822430260032214034568A5435C
:107390000C692C434460DB0304689C434B68234323
:1073A000036003680C24A3430C681C43046053026D
:1073B00004689C434B692343036012028368934330
:1073C0008A691A4382608968FFF7A4FFB0BD000094
:1073D000B0B51C480168022529430124A14301607E
:1073E00021052046FBF7B4FA17484168174A0A40BE
:1073F0001749511841602206014608390B681343AA
:107400000B600A689201FCD5210442680A4342607D
:1074100001682943052291430160016838220A402E
:10742000102AFAD107210A020368934303600A0372
:10743000036893430360090402688A430260FAF711
:10744000A3FCB0BD002002400810024006F8F9FF7E
:1074500061010200F8B516460D4604461F4F00288C
:1074600004D11F481F493A46FDF704F9002D04D105
:107470007A1C1DA01B49FDF7FDF81D4F3868002838
:1074800005D11648821C1B481649FDF7F3F8E06940
:10749000002805D11148C21C17A01249FDF7EAF8CF
:1074A000A169002901D02046884707202661606134
:1074B000102220462946FEF730FC3437F8F71AFE32
:1074C00039463F68002FFBD122462C320A60002546
:1074D000E562F8F713FE2846F8BDC0461305000024
:1074E00066950008959500086E616D6500000000C6
:1074F000841E0020729500086261636B656E642DC6
:107500003E6F75747075740080B500F011FA044810
:107510000449C16104A10122FFF79CFF002080BD46
:107520006C07002031750008636F6E736F6C650027
:1075300070B5049CFDF7FEF800280CD00546059BAD
:10754000068C402030432884002128462246FDF73F
:1075500035FA2E8470BD2046FDF78EFB70BD00000D
:10756000F0B587B002931746044601252E02002885
:10757000069105D152A054493246FDF77BF8069991
:10758000082904D3721C51484F49FDF773F80C9831
:10759000002F039005D1B21C4D484B49FDF76AF806
:1075A00003980197002804D1F21C4A484649FDF788
:1075B00061F804960D980090474E002005903060C9
:1075C0004648FEF790FB7060A6270699CF402F40F3
:1075D000306810D10D462118414A00F0C9F93168D0
:1075E00008183060A9003F4A5258211800F0C0F92D
:1075F0003168081830605B2121542018451CFFF7C2
:1076000017F80146284600F0D7F9316840180019EC
:107610005D224270059A82706018FEF764FB316843
:10762000081830602118304A304DA84731680818D2
:1076300030602118069A92002DA39A58A847316805
:10764000081830602118019AA8473168081830607E
:1076500021182F4AA8473168091831606018049D25
:10766000691A039A009BFFF7E7F901463068401852
:107670006A1C904200D30498002900DA0498306014
:1076800071680A18FC3A234B9A4202D8FB20401A30
:1076900030600299002906D02118104A00F068F9DC
:1076A000316808183060002F06D121181AA200F0A6
:1076B0005FF93168081830600599215407B0F0BDB2
:1076C0006C6F675F62756600879500084E950008CD
:1076D0006E950008C3950008A40100203C950008A1
:1076E00063950008F07C00088F8500087179000818
:1076F0003F950008000000000000000045950008CC
:107700004B950008000000004895000842950008CD
:107710008E850008FEFEFFFF1B5B306D0000000041
:10772000F0B58DB0099317460A910290FEF7DBFA87
:1077300004466B480068002804D16A486AA16E4A72
:10774000FCF798FFFBF720FD0546FCF7F1FD083438
:1077500003942C460120000206900026049635462C
:1077600008940998854200D3B5E0002D08D003980D
:1077700004994618202120463246FDF7FBFC2DE0F7
:107780005B20A05508988419601C0790FEF750FFF5
:107790000146079800F010F93018089940185D214B
:1077A0004170202181700021C1702046FEF79BFAB4
:1077B0000490841908980119204650A2514EB047F0
:1077C0002418089801192046029AB04724180898EE
:1077D000011920464C4AB0472618089C0A982818D8
:1077E0000590401E0090A019069C214647A22B46FA
:1077F000FEF76EFAA04200D8841900260A98B0421B
:1078000021D0A8190999884206D2BB5D0BA808218E
:1078100042A2FEF75DFA04E00BA808223EA1FEF7A3
:107820007CFA089801190BAA204600F0A1F8041967
:10783000761C7007E2D1089801192046394A00F0F9
:1078400097F80419DAE7079708980119204636A235
:1078500000F08EF8041900270A98B84219D0E819E8
:107860000999884213D20798C35D184620385F28CB
:1078700000D32E230BAE082130462CA2FEF728FAA7
:10788000089801192046324600F072F804197F1C4E
:10789000E2E7874E3046FEF726FA0019069988423D
:1078A00004D93046FEF71FFA06990C1A089D2919CB
:1078B0002046324600F05CF806192C460021A955F6
:1078C0000096072001222B46FBF77AF8079F0A98BB
:1078D0003F18059D45E7FCF745FD0DB0F0BDC046DE
:1078E000841E002072950008756C6F675F6865786C
:1078F00064756D7000000000E6020000442F4845EA
:1079000058200000717900088E8500082530345811
:107910002D253034583A20002020200025303258C0
:10792000200000008F850008202000002563000053
:10793000B0B5084D286800280AD12846083006A1AD
:1079400001242246FDF738FC002068632C606C603F
:107950000020B0BD841E0020756C6F670000000021
:107960001CB504AC0194009400F046F81CBD000066
:1079700070B514460D460646002904D10BA00C49EB
:107980009222FCF777FE002C04D10AA0084993222A
:10799000FCF770FE0020215C002905D03218FF2A78
:1079A00002D82954401CF6E770BDC04664737400C9
:1079B000D795000873726300F8B50E46054600249B
:1079C0000A2730463946F8F7A7FC4743F11B302217
:1079D0000A432A55641C092E0646F1D80020285572
:1079E000611E884206D22A5C6B5C2B546A54491E85
:1079F000401CF6E72046F8BDF0B585B01F4604925E
:107A00000C4606468D208500002904D122482349D2
:107A10002A46FCF72FFE002F04D16A1C20481F497C
:107A2000FCF728FE082E04D3EA1C1E481B49FCF76D
:107A300021FE1D48006800282BD00A9DFBF7A4FBFF
:107A40000390FCF775FC1949087801280AD13846DB
:107A50002946FDF731FA0498012818D11448FDF79A
:107A60002BFA14E00120087000970195039F384617
:107A700031462246049BFFF773FD009000253046F7
:107A800021462A463B46FAF79BFF08480570FCF75B
:107A900069FC05B0F0BDC0466E950008CA950008A7
:107AA000C39500084E950008841E0020C8200020C1
:107AB0003C950008B0B51048046810492046F8F716
:107AC0002BFC0F4D68607D20C1002046F8F724FC98
:107AD0002860EFF31084EFF3108072B6FBF764FBBD
:107AE000084DE961A861FBF75FFBE969A969401AE4
:107AF000286084F31088B0BD0C00002040420F00C5
:107B000004000020B001002080B5FEF78BF80020B3
:107B100080BD0000004870470000002002E008C857
:107B2000121F08C1002AFAD170477047002001E0F7
:107B300001C1121F002AFBD1704700404040404065
:107B40004040404041414141414040404040404030
:107B50004040404040404040404040050202020258
:107B6000020202020202020202020220202020205F
:107B70002020202020020202020202029090909017
:107B800090901010101010101010101010101010F5
:107B90001010101010100202020202028888888859
:107BA0008888080808080808080808080808080855
:107BB0000808080808080202020240003B7B00088F
:107BC00000000000000054545220524547474553DE
:107BD000000000010002000100030001000200019A
:107BE0000004000100020001000300010002000186
:107BF0000005000100020001000300010002000175
:107C00000004000100020001000300010002000165
:107C10000006000100020001000300010002000153
:107C20000004000100020001000300010002000145
:107C30000005000100020001000300010002000134
:107C40000004000100020001000300010002000125
:107C50000007000100020001000300010002000112
:107C60000004000100020001000300010002000105
:107C700000050001000200010003000100020001F4
:107C800000040001000200010003000100020001E5
:107C900000060001000200010003000100020001D3
:107CA00000040001000200010003000100020001C5
:107CB00000050001000200010003000100020001B4
:107CC00000040001000200010003000100020001A5
:107CD000000000003D2700084D280008E5270008A7
:107CE0000000000000000000000000000000000094
:107CF000839500080000000000000000AC8500082B
:107D00007F95000800000000B48500080000000016
:107D1000A98B0008708B0008038B0008158B0008E6
:107D20002B8B0008F68A0008458B0008368B00086C
:107D3000F38B0008528B00080C8C0008FB8B0008AA
:107D4000208B0008038C00088B8B0008DD8B00085B
:107D50007D8B00089C8B0008C88B0008BA8B00083C
:107D6000638B0008EB8B000801000000020000009C
:107D700004000000080000001000000020000000C7
:107D80004000000080000000000100018000800031
:107D9000800080000100030302020202017B78766A
:107DA0007472707E00F6000800F0000800EC000815
:107DB00000E8000800E4000800E0000800FC0008FB
:107DC0005F5F636D645F53797374656D5F52657354
:107DD0006574002253797374656D5F5265736574C1
:107DE00022005F5F636D645F4253505F5274635F54
:107DF0004461746554696D655F4366670022204283
:107E00004344E6A0BCE5BC8FE8BE93E585A52052BF
:107E10005443E697A5E69C9FE697B6E997B4E985B3
:107E20008DE7BDAE3A792C6D2C642C682C6D2C73CB
:107E30002C772022005F5F636D645F544553545F6D
:107E4000466C6173685F57726974655F5265636FF2
:107E500072640022544553545F466C6173685F57E7
:107E6000726974655F5265636F726422005F5F635D
:107E70006D645F544553545F466C6173685F52652F
:107E800061645F5265636F72640022544553545FAE
:107E9000466C6173685F526561645F5265636F72BF
:107EA00064220068656C6C6F007361792068656C92
:107EB0006C6F20776F726C640076657273696F6E99
:107EC0000073686F772052542D5468726561642086
:107ED00076657273696F6E20696E666F726D61741C
:107EE000696F6E005F5F636D645F76657273696F63
:107EF0006E0073686F772052542D54687265616408
:107F00002076657273696F6E20696E666F726D613F
:107F100074696F6E006C6973745F74687265616414
:107F2000006C69737420746872656164005F5F63DC
:107F30006D645F6C6973745F746872656164006C12
:107F400069737420746872656164006C6973745F2E
:107F500073656D006C6973742073656D6170686F13
:107F6000726520696E2073797374656D005F5F635D
:107F70006D645F6C6973745F73656D006C697374B5
:107F80002073656D6170686F726520696E2073790A
:107F90007374656D006C6973745F6576656E7400EB
:107FA0006C697374206576656E7420696E207379D0
:107FB0007374656D005F5F636D645F6C6973745F9C
:107FC0006576656E74006C697374206576656E7491
:107FD00020696E2073797374656D006C6973745FCA
:107FE0006D75746578006C697374206D757465784F
:107FF00020696E2073797374656D005F5F636D64D3
:108000005F6C6973745F6D75746578006C69737407
:10801000206D7574657820696E2073797374656D51
:10802000006C6973745F6D61696C626F78006C6974
:108030007374206D61696C20626F7820696E2073A3
:10804000797374656D005F5F636D645F6C697374F1
:108050005F6D61696C626F78006C697374206D612B
:10806000696C20626F7820696E2073797374656D16
:10807000006C6973745F6D73677175657565006C0D
:10808000697374206D6573736167652071756575BB
:108090006520696E2073797374656D005F5F636D31
:1080A000645F6C6973745F6D736771756575650086
:1080B0006C697374206D6573736167652071756594
:1080C000756520696E2073797374656D006C6973D2
:1080D000745F74696D6572006C6973742074696D86
:1080E000657220696E2073797374656D005F5F63DC
:1080F0006D645F6C6973745F74696D6572006C693F
:1081000073742074696D657220696E20737973745D
:10811000656D006C6973745F646576696365006C96
:108120006973742064657669636520696E2073796C
:108130007374656D005F5F636D645F6C6973745F1A
:10814000646576696365006C69737420646576693B
:10815000636520696E2073797374656D006C697353
:1081600074006C69737420616C6C2073796D626F3C
:108170006C20696E2073797374656D005F5F636D49
:10818000645F68656C700052542D54687265616458
:10819000207368656C6C2068656C702E005F5F638F
:1081A0006D645F7073004C697374207468726561EC
:1081B000647320696E207468652073797374656DCB
:1081C0002E005F5F636D645F667265650053686F64
:1081D0007720746865206D656D6F727920757361A5
:1081E000676520696E207468652073797374656DA6
:1081F0002E006C6973745F6D656D006C697374201B
:108200006D656D6F727920757361676520696E6643
:108210006F726D6174696F6E0000000000000000F5
:1082200000000050010000000100000000000050AC
:1082300002000000020000000000005004000000E6
:1082400003000000000000500800000004000000CF
:108250000000005010000000050000000000005069
:108260002000000006000000000000504000000058
:10827000070000000000005080000000080000001F
:108280000000005000010000090000000000005044
:10829000000200000A00000000000050000400007E
:1082A0000B00000000000050000800000C0000005F
:1082B00000000050001000000D0000000000005001
:1082C000002000000E0000000000005000400000F0
:1082D0000F000000000000500080000010000000AF
:1082E00000040050010000001100000000040050D4
:1082F0000200000012000000000400500400000012
:1083000013000000000400500800000014000000EA
:108310000004005010000000150000000004005090
:108320002000000016000000000400504000000083
:10833000170000000004005080000000180000003A
:10834000000400500001000019000000000400506B
:10835000000200001A0000000004005000040000A9
:108360001B00000000040050000800001C0000007A
:1083700000040050001000001D0000000004005028
:10838000002000001E00000000040050004000001B
:108390001F000000000400500080000020000000CA
:1083A00000080050010000002100000000080050FB
:1083B000020000002200000000080050040000003D
:1083C0002300000000080050080000002400000006
:1083D00000080050100000002500000000080050B8
:1083E00020000000260000000008005040000000AF
:1083F0002700000000080050800000002800000056
:108400000008005000010000290000000008005092
:10841000000200002A0000000008005000040000D4
:108420002B00000000080050000800002C00000095
:1084300000080050001000002D000000000800504F
:10844000002000002E000000000800500040000046
:108450002F000000000800500080000030000000E5
:10846000000C00500100000031000000000C005022
:108470000200000032000000000C00500400000068
:1084800033000000000C0050080000003400000021
:10849000000C00501000000035000000000C0050DF
:1084A0002000000036000000000C005040000000DA
:1084B00037000000000C0050800000003800000071
:1084C000000C00500001000039000000000C0050BA
:1084D000000200003A000000000C00500004000000
:1084E0003B000000000C0050000800003C000000B1
:1084F000000C0050001000003D000000000C005077
:10850000002000003E000000000C00500040000071
:108510003F000000000C0050008000006B416C61C7
:10852000726D5265636F726428256429006B466121
:10853000756C745265636F726428256429006B4101
:108540006C61726D5263795265636F726428256441
:1085500029006B4661756C745263795265636F7262
:1085600064282564290068725F72785F73656D0006
:108570006273705F6872006B4E756D4F6652656313
:108580006F72647300443A2000453A2000493A2053
:10859000006273705F666C617368001B5B313B3314
:1085A000306D001B5B306D001B5B313B33316D0068
:1085B0001B5B313B33326D002020257325737265C0
:1085C0006164203A68725F73746172745F6164649D
:1085D00072203D202523782C20696E6465785F61C8
:1085E0006464723A202523782C2068725F6E756D62
:1085F0003A2025642C2068725F706167653A2564B3
:108600002C20726561645F64617461203A202025CA
:1086100023580D0A0D0A2573002020257325734663
:108620006C6173685F4765744D61784E756D28287D
:108630002564295F5265636F72647328256429205D
:1086400053756D5F436865636B2825235829202186
:108650003D20636865636B5F73756D28252358291A
:108660002C696E6465785F61646472203A252358D2
:108670000D0A0D0A257300202025732573466C61B1
:1086800073685F45726173655061676520666169F3
:108690006C65640D0A0D0A2573002020257325736F
:1086A000466163746F727954696D652063686563B0
:1086B0006B5F73756D206572726F720D0A0D0A25FE
:1086C0007300202025732573457870697261746981
:1086D0006F6E54696D65206973206E6F74207365C9
:1086E000740D0A0D0A257300202025732573466139
:1086F00063746F727954696D65206973206E6F744D
:10870000207365740D0A0D0A25730020202573253A
:1087100073466C6173685F57726974655F2825647E
:10872000295265636F726428256429206E756D2057
:108730003E3D207265636F72646564204D617820F0
:108740006E756D282564290D0A2573002020257378
:10875000257372656164203A68725F737461727424
:108760005F61646472203D202523782C20696E644B
:1087700065785F616464723A202523782C206872E2
:108780005F6E756D3A2025642C2068725F7061679A
:10879000653A25642C20726561645F6461746120B0
:1087A0003A20202523580D0A257300202025732503
:1087B00073466C6173685F4572617365506167658C
:1087C0005F5265636F726473206661696C656420D3
:1087D00065726173655F706167653A202523582073
:1087E000213D20202523580D0A25730020202573C4
:1087F000257377726974653A68725F737461727415
:108800005F61646472203D202523782C20696E64AA
:1088100065785F616464723A202523782C20687241
:108820005F6E756D3A2025642C2068725F706167F9
:10883000653A25642C2077726974655F64617461A0
:10884000203A202523580D0A257300202025732562
:108850007368725F73746172745F61646472203DE7
:10886000202523782C20696E6465785F61646472CA
:108870003A202523782C2068725F6E756D3A20258A
:10888000642C2068725F706167653A25642C2077DC
:10889000726974655F64617461203A202523580D04
:1088A0000A257300202025732573466C6173685F69
:1088B00057726974655F282564295265636F726415
:1088C0003A253034642D253032642D253032642031
:1088D000253032643A253032642C20636865636B3E
:1088E0005F73756D203A202523580D0A25730020EB
:1088F0002025732573496E6465785F4672616D65E6
:108900002E68725F696E6465785F61646472203D91
:108910002068725F73746172745F616464725B7209
:1089200065636F72645D202B2069202A20464C41CC
:1089300053485F504147455F425954455F53495A38
:1089400045202D2048525F5245434F52445F4652C6
:10895000414D455F4C454E203D202523580D0A25AD
:108960007300202025732573457261736520506163
:1089700067652025640D0A25730020202573257363
:10898000696E646578206E756D2028256429203E07
:108990002041637475616C2073746F726167652028
:1089A0006E756D2025640D0A257300202025732522
:1089B00073466C6173685F526561642044617461E1
:1089C000204D69736D617463682061742061646413
:1089D00072202523582C20657870656374656420A7
:1089E000256420676F742025640D0A2573002020FC
:1089F00025732573466C6173685F526561645F28F7
:108A00002564295265636F7264282564293A2530EC
:108A100034642D253032642D253032642C253032DB
:108A2000643A253032640D0A257300202025732511
:108A300073466C6173685F526561645F466163741D
:108A40006F727954696D653A253034642D25303262
:108A5000642D253032642C253032643A253032645E
:108A60000D0A25730020202573257372656164202B
:108A70003A68725F73746172745F61646472322009
:108A80003D202523780D0A257300646561637469B0
:108A900076617465640A00252D2A2E732070726930
:108AA000202073746174757320202020202073703F
:108AB0002020202020737461636B2073697A652005
:108AC0006D61782075736564206C656674207469C7
:108AD000636B20206572726F720A0020696E697480
:108AE0002020200020636C6F7365202000207265B9
:108AF00061647920200052544300207375737065BF
:108B00006E64004E6574776F726B20496E74657287
:108B100066616365004D5444204465766963650071
:108B2000535049204465766963650043414E2044B3
:108B300065766963650047726170686963204465A2
:108B40007669636500536F756E642044657669636A
:108B5000650055534220536C617665204465766903
:108B6000636500546F7563682044657669636500CA
:108B7000426C6F636B2044657669636500506F7269
:108B800074616C2044657669636500504D205073B4
:108B90006575646F204465766963650054696D6529
:108BA000722044657669636500436861726163742D
:108BB0006572204465766963650053656E736F72F4
:108BC00020446576696365004D697363656C6C610B
:108BD0006E656F75732044657669636500506970D2
:108BE00065002072756E6E696E6700556E6B6E6FF4
:108BF000776E00493243204275730053504920423A
:108C00007573005344494F204275730055534220F9
:108C1000486F737420427573005F5F636D645F001B
:108C200008007368656C6C20213D2052545F4E55DE
:108C30004C4C00256300257325730072745F7468C3
:108C4000726561645F69646C655F6578637574659E
:108C50000046756E6374696F6E5B25735D20736883
:108C6000616C6C206E6F7420626520757365642082
:108C7000696E204953520A0046756E6374696F6EBF
:108C80005B25735D207368616C6C206E6F7420626D
:108C9000652075736564206265666F726520736315
:108CA000686564756C65722073746172740A007310
:108CB000697A6520213D2030006D6220213D2052DF
:108CC000545F4E554C4C0073656D20213D2052542D
:108CD0005F4E554C4C006D7120213D2052545F4E2B
:108CE000554C4C0062756666657220213D205254D9
:108CF0005F4E554C4C006576656E7420213D2052C8
:108D0000545F4E554C4C006D7574657820213D20A4
:108D100052545F4E554C4C0076616C7565203C207A
:108D200030783130303030550072745F6576656E62
:108D3000745F73656E640072745F73656D5F7461F8
:108D40006B650072745F6D757465785F74616B65D7
:108D50000072745F6F626A6563745F6765745F74E5
:108D6000797065282673656D2D3E706172656E742D
:108D70002E706172656E7429203D3D2052545F4F04
:108D8000626A6563745F436C6173735F53656D61A1
:108D900070686F72650072745F73656D5F72656C89
:108DA000656173650072745F6D757465785F726577
:108DB0006C656173650072745F6D625F637265619B
:108DC00074650072745F73656D5F6372656174656D
:108DD0000072745F6D715F637265617465007274B7
:108DE0005F6576656E745F63726561746500727449
:108DF0005F6D757465785F63726561746500727428
:108E00005F6D625F64656C6574650072745F736545
:108E10006D5F64656C6574650072745F6D715F642D
:108E2000656C6574650072745F6576656E745F6409
:108E3000656C6574650072745F6D757465785F64E8
:108E4000656C6574650072745F6F626A6563745FF8
:108E50006765745F7479706528266D712D3E706149
:108E600072656E742E706172656E7429203D3D20AE
:108E700052545F4F626A6563745F436C6173735FE2
:108E80004D65737361676551756575650072745FD3
:108E90006D625F6465746163680072745F73656DB1
:108EA0005F6465746163680072745F6D715F6465AF
:108EB000746163680072745F6576656E745F646583
:108EC000746163680072745F6D757465785F646562
:108ED000746163680072745F6D625F636F6E747259
:108EE0006F6C0072745F73656D5F636F6E74726F29
:108EF0006C0072745F6D715F636F6E74726F6C0083
:108F000072745F6576656E745F636F6E74726F6C9A
:108F10000072745F6D757465785F636F6E74726FE5
:108F20006C0072745F6D625F73656E645F77616918
:108F3000740072745F6D715F73656E645F776169F1
:108F4000740072745F73656D5F696E69740072742A
:108F50005F6D715F757267656E740072745F6F62CA
:108F60006A6563745F6765745F74797065282665E8
:108F700076656E742D3E706172656E742E706172CE
:108F8000656E7429203D3D2052545F4F626A6563CF
:108F9000745F436C6173735F4576656E74007274C1
:108FA0005F6D625F726563760072745F6D715F7290
:108FB0006563760072745F6576656E745F72656373
:108FC000760072745F6F626A6563745F6765745F71
:108FD0007479706528266D757465782D3E706172A0
:108FE000656E742E706172656E7429203D3D20524D
:108FF000545F4F626A6563745F436C6173735F4D66
:10900000757465780072745F6F626A6563745F6718
:1090100065745F7479706528266D622D3E7061728B
:10902000656E742E706172656E7429203D3D20520C
:10903000545F4F626A6563745F436C6173735F4D25
:1090400061696C426F78002872745F756261736544
:109050005F7429282872745F75696E74385F742094
:109060002A296D656D202B2053495A454F465F5381
:1090700054525543545F4D454D2920252052545F8D
:10908000414C49474E5F53495A45203D3D203000F1
:109090006D656D2D3E6D61676963203D3D204845DE
:1090A00041505F4D414749430072745F7265616C86
:1090B0006C6F630072745F6D616C6C6F630028721B
:1090C000745F75696E74385F74202A29726D656DDE
:1090D000203E3D202872745F75696E74385F74207D
:1090E0002A29686561705F707472202626202872B4
:1090F000745F75696E74385F74202A29726D656DAE
:10910000203C202872745F75696E74385F74202A61
:1091100029686561705F656E64002872745F7562AE
:109120006173655F74296D656D202B2053495A4525
:109130004F465F5354525543545F4D454D202B20AD
:1091400073697A65203C3D202872745F7562617393
:10915000655F7429686561705F656E640072745F35
:109160006672656500706C75675F686F6C6573002B
:1091700072745F73797374656D5F686561705F6940
:109180006E697400696E666F726D6174696F6E20CE
:10919000213D2052545F4E554C4C006F626A65630E
:1091A0007420213D2052545F4E554C4C0072745F28
:1091B0006F626A6563745F66696E640072745F6F84
:1091C000626A6563745F616C6C6F63617465007281
:1091D000745F6F626A6563745F64656C6574650073
:1091E00072745F6F626A6563745F696E697400743C
:1091F000687265616420213D2052545F4E554C4C8D
:109200000072745F6F626A6563745F6765745F7430
:10921000797065282872745F6F626A6563745F7421
:109220002974687265616429203D3D2052545F4F66
:10923000626A6563745F436C6173735F54687265DF
:1092400061640072745F7468726561645F737573E2
:1092500070656E640072745F7468726561645F72D9
:109260006573756D650072745F7468726561645FC3
:1092700064656C6574650072745F746872656164BE
:109280005F6465746163680072745F7468726561BD
:10929000645F64656C61795F756E74696C0072748B
:1092A0005F7468726561645F636F6E74726F6C0087
:1092B00072745F7468726561645F736C6565700079
:1092C00072745F7468726561645F737461727475DF
:1092D000700072745F7468726561645F696E69744E
:1092E0000072745F7468726561645F74696D656F44
:1092F00075740074696D657220213D2052545F4E73
:10930000554C4C0072745F74696D65725F64656C76
:109310006574650072745F74696D65725F6465740D
:109320006163680072745F74696D65725F636F6E0C
:1093300074726F6C0072745F74696D65725F7374C0
:109340006F700072745F6F626A6563745F676574E3
:109350005F74797065282674696D65722D3E706141
:1093600072656E7429203D3D2052545F4F626A65DC
:1093700063745F436C6173735F54696D65720072EF
:10938000745F74696D65725F737461727400646593
:109390007620213D2052545F4E554C4C00546F2096
:1093A000696E697469616C697A6520646576696360
:1093B000653A2573206661696C65642E2054686582
:1093C000206572726F7220636F6465206973202557
:1093D000640072745F6465766963655F7265616479
:1093E0000072745F6F626A6563745F6765745F744F
:1093F00079706528266465762D3E706172656E749D
:1094000029203D3D2052545F4F626A6563745F437B
:109410006C6173735F446576696365006B65726E3A
:10942000656C2E6465766963650072745F64657649
:109430006963655F636C6F73650072745F64657602
:109440006963655F7365745F72785F696E64696391
:109450006174650072745F6465766963655F7365E6
:10946000745F74785F636F6D706C6574650072749F
:109470005F6465766963655F7772697465007274AD
:109480005F6465766963655F636F6E74726F6C00AD
:1094900072745F6465766963655F6F70656E007294
:1094A000745F6465766963655F756E72656769731D
:1094B0007465720072745F6465766963655F646584
:1094C0007374726F790070696E20213D2052545F71
:1094D0004E554C4C005F68775F70696E2E6F7073ED
:1094E00020213D2052545F4E554C4C0020202573C6
:1094F0002573737461727475702075617274315F55
:10950000646D615F72785F74687265616420726512
:109510007475726E203D2025640D0A257300555325
:109520004152543120496E6974006472765F7561EE
:109530007274005465726D696E616C000D0A0041B1
:109540002F00442F00452F00492F00572F006C6536
:1095500076656C203C3D204C4F475F4C564C5F4439
:109560004247001B5B006261636B656E640074615F
:109570006700756C6F672E696E69745F6F6B00337F
:10958000336D0033356D00756C6F675F666F726D9C
:109590006174657200756C6F675F6261636B656EA5
:1095A000645F726567697374657200756C6F675F7D
:1095B0006261636B656E645F756E72656769737413
:1095C000657200666F726D617400756C6F675F76AF
:1095D0006F757470757400756C6F675F7374726308
:1095E00070790000796D0008716D0008754D0008F4
:1095F000317900086D6D000855070008D123000877
:10960000ED4D00080975000891050008B106000835
:109610007D2C000861260008756D0008C07D0008DB
:10962000D37D00082D1E0008E27D0008FD7D0008A6
:10963000E5070008357E0008537E0008A51E0008D7
:109640006D7E00088A7E0008311E0008A37E000897
:10965000A97E0008F1310008B97E0008C17E00082B
:10966000097B0008E47E0008F27E0008097B000800
:10967000157F0008217F0008B53A00082D7F0008FB
:109680003F7F0008B53A00084B7F0008547F000870
:10969000893900086D7F00087C7F0008893900083F
:1096A000957F0008A07F0008E5330008B57F00081B
:1096B000C67F0008E5330008DB7F0008E67F00086E
:1096C00079380008FB7F00080C8000087938000812
:1096D000218000082E800008893500084680000897
:1096E0005980000889350008718000087F800008D3
:1096F000453700089C800008B08000084537000806
:10970000CD800008D88000082D3C0008ED800008BE
:10971000FE8000082D3C0008138100081F8100080E
:10972000D93200083581000847810008D932000885
:109730005D810008628100086D3200087C810008AC
:1097400087810008954200089D810008A6810008D5
:10975000B7290008C2810008CD810008AD290008A2
:10976000F2810008FB810008D936000890970008B4
:1097700000000020900000001C7B000820980008DA
:1097800090000020402400002C7B00088D8EFFFFFD
:109790000000000001000000010000000024F400AF
:1097A00001000000140000201400002090000000C0
:1097B00002000000240000202400002028000000F7
:1097C0000300000034000020340000202C000000C2
:1097D0000400000044000020440000202800000095
:1097E0000500000054000020540000203800000054
:1097F0000600000064000020640000204400000017
:1098000009000000740000207400002048000000DF
:109810000A000000840000208400002034000000C2
:04000005080000C12E
:00000001FF
